:020000040000FA
:0400000007EF00F016
:100008007882B1ED1EF078EF4AF0F2EC52F0000E73
:100018000D6E000E93EC51F069EF04F0D20E106EE5
:10002800F90E116EF7EC48F0010E0D6E020E93EC0E
:1000380051F0830E106EFD0E116EF7EC48F0C5EF0F
:1000480004F0BF0E106EF90E116EF7EC48F0010EB9
:100058000D6E010E93EC51F0D50E106EFE0E116E62
:10006800F7EC48F057C115F058C116F0040E176E9A
:10007800010E186E57EC3EF0010E0D6E020E93EC59
:1000880051F0CD0E106EFF0E116EF7EC48F05BC10B
:1000980015F05CC116F0040E176E010E186E57ECC1
:1000A8003EF0870E106EFF0E116EF7EC48F05DC142
:1000B80015F05EC116F0040E176E010E186E57EC9F
:1000C8003EF0010E0D6E030E93EC51F0430E106ED0
:1000D800FF0E116EF7EC48F059C108F05AC109F04B
:1000E800000E0B6E0A0E0A6E51EC40F008C027F0A5
:1000F80009C028F027C008F028C009F0000E0B6ED0
:100108000A0E0A6E98EC52F0081E091E084A092ABF
:10011800010159510824256E5A510920266E27C01D
:1001280015F028C016F0010E176E010E186EAAEC15
:1001380041F02E0E05EC4BF025C015F026C016F048
:10014800010E176E010E186EAAEC41F0C5EF04F00F
:10015800AF0E106EFB0E116EF7EC48F0010E0D6E2F
:10016800020E93EC51F06FC11BF070C11CF071C10D
:100178001DF072C11EF0060E1F6E010E206EF7EC08
:1001880030F0C5EF04F0F50E106EF70E116EF7ECB7
:1001980048F0010E0D6E020E93EC51F001015F5113
:1001A800D8B4D9EF00F0DBEF00F0E3EF00F0240E55
:1001B800106EFD0E116EF7EC48F0C5EF04F0670EF7
:1001C800106EFD0E116EF7EC48F0C5EF04F0C5EFA8
:1001D80004F0EA0E106EFD0E116EF7EC48F0010EF9
:1001E8000D6E020E93EC51F0770E106EFD0E116E2F
:1001F800F7EC48F060C115F061C116F0030E176EF8
:10020800010E186EAAEC41F0C5EF04F0640E106EF2
:10021800F70E116EF7EC48F0010E0D6E020E93EC1E
:1002280051F001017351D8B41CEF01F01EEF01F039
:1002380026EF01F0DF0E106EFD0E116EF7EC48F0A0
:10024800C5EF04F0D40E106EFD0E116EF7EC48F0F9
:10025800C5EF04F0C5EF04F0120E106EFB0E116E20
:10026800F7EC48F0010E0D6E020E93EC51F001010F
:100278007451D8B442EF01F044EF01F04CEF01F0B3
:10028800810E106EFF0E116EF7EC48F0C5EF04F00A
:10029800C80E106EFF0E116EF7EC48F0C5EF04F0B3
:1002A800C5EF04F03F0E106EFC0E116EF7EC48F02F
:1002B800010E0D6E020E93EC51F075C108F076C177
:1002C80009F0000E0B6E0A0E0A6E91EC4BF008C096
:1002D80027F009C028F027C008F028C009F0000E50
:1002E8000B6E0A0E0A6E98EC52F0081E091E084A98
:1002F800092A010175510824256E76510920266EB8
:1003080027C015F028C016F0010E176E010E186EE2
:10031800AAEC41F02E0E05EC4BF025C015F026C0D6
:1003280016F0010E176E010E186EAAEC41F0C5EF1B
:1003380004F0430E106EFD0E116EF7EC48F001014B
:100348007851D8A4AAEF01F0ACEF01F0C4EF01F0A6
:10035800010E0D6E010E93EC51F0E20E106EFC0EC4
:10036800116EF7EC48F0010E0D6E020E93EC51F091
:10037800D40E106EFC0E116EF7EC48F0C5EF04F0C9
:10038800010E0D6E010E93EC51F0C60E106EFC0EB0
:10039800116EF7EC48F0010E0D6E020E93EC51F061
:1003A800F00E106EFC0E116EF7EC48F0C5EF04F07D
:1003B800C5EF04F03A0E106EF70E116EF7EC48F028
:1003C800010E0D6E020E93EC51F00001BFAFEFEF7E
:1003D80001F0F1EF01F0F9EF01F0E10E106EFF0E00
:1003E800116EF7EC48F0C5EF04F00001BF51216E23
:1003F800226A6950211807E16A502218D8A407EF29
:1004080002F009EF02F011EF02F0C30E106EFF0EBA
:10041800116EF7EC48F0C5EF04F09F0E106EFB0E5E
:10042800116EF7EC48F00001BF51310F05EC4BF0AD
:10043800290E05EC4BF0C5EF04F0C5EF04F0C5EF4D
:1004480004F06C0E106EFB0E116EF7EC48F0010E06
:100458000D6E020E93EC51F0240E106EFB0E116E11
:10046800F7EC48F0C5EF04F0DC0E106EFA0E116ED2
:10047800F7EC48F0010E0D6E020E93EC51F00001FE
:10048800C0AF49EF02F04BEF02F053EF02F0F50E68
:10049800106EFF0E116EF7EC48F0C5EF04F08D0EEC
:1004A800106EFF0E116EF7EC48F00001C051300FCE
:1004B80005EC4BF05D0E05EC4BF0C5EF04F0C5EF15
:1004C80004F0F2EC52F0000E0D6E000E93EC51F0B9
:1004D8004E0E106EFC0E116EF7EC48F0000E0D6E0D
:1004E800010E93EC51F04A0E106EFF0E116EF7ECF0
:1004F80048F0000E0D6E020E93EC51F0580E106E7F
:10050800FF0E116EF7EC48F0000E0D6E030E93EC23
:1005180051F08E0E106EF70E116EF7EC48F0C5EF25
:1005280004F0790E106EF70E116EF7EC48F0010E1C
:100538000D6E020E93EC51F0010179AFA6EF02F0B7
:10054800A8EF02F0B0EF02F0C30E106EFF0E116EAE
:10055800F7EC48F0C5EF04F0E10E106EFF0E116ED7
:10056800F7EC48F0C5EF04F0C5EF04F0990E106EF3
:10057800F90E116EF7EC48F0010E0D6E020E93ECB9
:1005880051F001017AAFCBEF02F0CDEF02F0D5EFD9
:1005980002F0C30E106EFF0E116EF7EC48F0C5EFB7
:1005A80004F0E10E106EFF0E116EF7EC48F0C5EF87
:1005B80004F0C5EF04F0AC0E106EF90E116EF7ECF6
:1005C80048F0010E0D6E010E93EC51F0D50E106E31
:1005D800FE0E116EF7EC48F07BC115F07CC116F0E9
:1005E800040E176E010E186E57EC3EF0010E0D6EDC
:1005F800020E93EC51F0CD0E106EFF0E116EF7EC5B
:1006080048F07FC115F080C116F0040E176E010E78
:10061800186E57EC3EF0870E106EFF0E116EF7EC59
:1006280048F081C115F082C116F0040E176E010E54
:10063800186E57EC3EF0010E0D6E030E93EC51F060
:10064800430E106EFF0E116EF7EC48F07DC108F0F6
:100658007EC109F0000E0B6E0A0E0A6E51EC40F0D6
:1006680008C027F009C028F027C008F028C009F002
:10067800000E0B6E0A0E0A6E98EC52F0081E091E48
:10068800084A092A01017D510824256E7E51092056
:10069800266E27C015F028C016F0010E176E010E41
:1006A800186EAAEC41F02E0E05EC4BF025C015F0A3
:1006B80026C016F0010E176E010E186EAAEC41F056
:1006C800C5EF04F0E10E106EF70E116EF7EC48F06E
:1006D800010E0D6E020E93EC51F0CD0E106EFE0E53
:1006E800116EF7EC48F083C115F084C116F0060EC0
:1006F800176E010E186E57EC3EF0C5EF04F0EE0EC3
:10070800106EFA0E116EF7EC48F0010E0D6E020E27
:1007180093EC51F08AC115F08BC116F0050E176ED7
:10072800010E186EAAEC41F0C5EF04F04F0E106EE2
:10073800F70E116EF7EC48F0010E0D6E020E93ECF9
:1007480051F001018651D8B4ACEF03F0AEEF03F0DD
:10075800B6EF03F0DF0E106EFD0E116EF7EC48F0E9
:10076800C5EF04F0D40E106EFD0E116EF7EC48F0D4
:10077800C5EF04F0C5EF04F0000E106EFB0E116E0D
:10078800F7EC48F0010E0D6E020E93EC51F00101EA
:100798008551D8B4D2EF03F0D4EF03F0DCEF03F0C7
:1007A800E50E106EFE0E116EF7EC48F0C5EF04F082
:1007B800730E106EFE0E116EF7EC48F0C5EF04F0E4
:1007C800C5EF04F0250E106EF70E116EF7EC48F029
:1007D800010E0D6E020E93EC51F001018751D8B451
:1007E800F8EF03F0FAEF03F002EF04F0810E106E59
:1007F800FF0E116EF7EC48F0C5EF04F0C80E106E4E
:10080800FF0E116EF7EC48F0C5EF04F0C5EF04F0E9
:100818008CC108F08DC109F0000E0B6E640E0A6ED3
:1008280091EC4BF008C023F009C024F0010E0D6EC6
:10083800020E93EC51F023C015F024C016F0020EFE
:10084800176E010E186E57EC3EF08D0E106EFD0EF1
:10085800116EF7EC48F023C008F024C009F0000E30
:100868000B6E640E0A6E98EC52F0081E091E084AB8
:10087800092A01018C510824236E8D510920246E08
:1008880023C015F024C016F0020E176E000E186E65
:1008980057EC3EF0E50E106EFF0E116EF7EC48F0C7
:1008A800490E106EFE0E116EF7EC48F0000E0D6E3C
:1008B800000E93EC51F0BF0E106EFB0E116EF7ECAC
:1008C80048F0C5EF04F0C5EF04F00001A651000A96
:1008D800D8B425EF00F0010AD8B4ACEF00F0030A51
:1008E800D8B4C7EF00F0010AD8B4EDEF00F0070A5A
:1008F800D8B40AEF01F0010AD8B430EF01F0030AC6
:10090800D8B456EF01F0010AD8B4DEEF01F00F0AAF
:10091800D8B425EF02F0010AD8B438EF02F0030A80
:10092800D8B412EF00F0010AD8B495EF02F0070A24
:10093800D8B4BAEF02F0010AD8B4DFEF02F0030A24
:10094800D8B466EF03F0010AD8B483EF03F01F0AA6
:10095800D8B49AEF03F0010AD8B4C0EF03F0030A41
:10096800D8B40CEF04F0010AD8B4E6EF03F0070A94
:10097800D8B49DEF01F0010AD8B465EF02F0C5EFD5
:1009880004F012007450030D000EF324556E030E8C
:10099800F420566E20EE02F05550D9265650DA2231
:1009A800DF50506E5050526E516A20EE01F0555093
:1009B800D9265650DA22DF50536E53505124576EC1
:1009C800000E5220586E20EE01F05550D926565090
:1009D800DA22DF50546E9BEF08F0190E0001C3199C
:1009E800D8A4F9EF04F0FBEF04F0FFEF04F0000ED9
:1009F800C36F02EF05F0C32B02EF05F0000EC56FC1
:100A0800C5C0C4F0000E206E020E1F6E74C021F027
:100A1800226AC30E236E000E246E000E256E000E91
:100A2800266E0DEC0FF0D6EF08F00001C351D8A4E4
:100A380020EF05F022EF05F026EF05F0190EC36F41
:100A480029EF05F0C30729EF05F0000EC56FC5C0F3
:100A5800C4F0000E206E020E1F6E74C021F0226AD0
:100A6800C30E236E000E246E000E256E000E266E39
:100A78000DEC0FF0D6EF08F052EF05F052EF05F04D
:100A880052EF05F052EF05F052EF05F052EF05F086
:100A980052EF05F052EF05F052EF05F076500001E5
:100AA800AB19D8B45AEF05F05CEF05F079EF05F013
:100AB800D00E506EFF0E516E7650526E536A5050E3
:100AC800522651505322410E5224F66EEF0E5320F7
:100AD800F76EF86A000EF8220800F5CFC3F0000E92
:100AE800C56FC5C0C4F088EF05F0C32B190EC365E8
:100AF80080EF05F082EF05F088EF05F0000EC36F78
:100B080088EF05F088EF05F0000E206E020E1F6ECC
:100B180074C021F0226AC30E236E000E246E000EEC
:100B2800256E000E266E0DEC0FF0D6EF08F0000EC5
:100B3800206E020E1F6E74C021F0226AC30E236E4F
:100B4800000E246E000E256E010E266E0DEC0FF0C1
:100B5800000E0D6E000E93EC51F044EF08F057C0F4
:100B68004DF058C04EF00D0E4F6E4AEC50F04DC08F
:100B780057F04EC058F020EE01F05550D926565087
:100B8800DA2257C0DFFF20EE02F05550D926565022
:100B9800DA225850DF6E7CEF08F057C04DF058C08D
:100BA8004EF00D0E4F6E4AEC50F04DC057F04EC04F
:100BB80058F020EE01F05550D9265650DA2257C089
:100BC800DFFF20EE02F05550D9265650DA22585051
:100BD800DF6E7CEF08F057C04DF058C04EF00D0E98
:100BE8004F6E4AEC50F04DC057F04EC058F020EE12
:100BF80001F05550D9265650DA2257C0DFFF20EEB3
:100C080002F05550D9265650DA225850DF6E7CEF44
:100C180008F0E50E106EF80E116EF7EC48F057C0AC
:100C280008F058C009F0000E0B6E010E0A6E270E70
:100C38000D6E0F0E0C6EF5EC50F008C057F009C0A1
:100C480058F00F0E326E040E336E57C034F058C091
:100C580035F0630E366E020EEEEC15F032C057F02A
:100C680033C058F057C008F058C009F0000E0B6E9A
:100C7800010E0A6E270E0D6E0F0E0C6EF5EC50F07D
:100C880008C057F009C058F020EE01F05550D92699
:100C98005650DA2257C0DFFF20EE02F05550D92611
:100CA8005650DA225850DF6E7CEF08F0D10E106EE5
:100CB800F80E116EF7EC48F057C008F058C009F06C
:100CC800000E0B6E000E0A6E270E0D6E0F0E0C6EC8
:100CD800F5EC50F008C057F009C058F00E0E326E0F
:100CE800040E336E57C034F058C035F0630E366EBC
:100CF800020EEEEC15F032C057F033C058F057C072
:100D080008F058C009F0000E0B6E000E0A6E270E90
:100D18000D6E0F0E0C6EF5EC50F008C057F009C0C0
:100D280058F020EE01F05550D9265650DA2257C017
:100D3800DFFF20EE02F05550D9265650DA225850DF
:100D4800DF6E7CEF08F0D10E106EF80E116EF7EC26
:100D580048F057C008F058C009F0000E0B6E000E9E
:100D68000A6E270E0D6E0F0E0C6EF5EC50F008C0D3
:100D780057F009C058F00D0E326E040E336E57C08E
:100D880034F058C035F0630E366E020EEEEC15F0F6
:100D980032C057F033C058F057C008F058C009F0B7
:100DA800000E0B6E000E0A6E270E0D6E0F0E0C6EE7
:100DB800F5EC50F008C057F009C058F020EE01F0EB
:100DC8005550D9265650DA2257C0DFFF20EE02F0E0
:100DD8005550D9265650DA225850DF6E7CEF08F06D
:100DE800CD0E106EF60E116EF7EC48F057C008F0F5
:100DF80058C009F0000E0B6E010E0A6E030E0D6E40
:100E0800E70E0C6EF5EC50F008C057F009C058F02A
:100E18000D0E326E030E336E57C034F058C035F0E5
:100E2800630E366E020EEEEC15F032C057F033C08A
:100E380058F057C008F058C009F0000E0B6E010EAC
:100E48000A6E030E0D6EE70E0C6EF5EC50F008C03E
:100E580057F009C058F020EE01F05550D9265650E9
:100E6800DA2257C0DFFF20EE02F05550D92656503F
:100E7800DA225850DF6E7CEF08F06C0E106EFC0E14
:100E8800116EF7EC48F0010E086E050E096E54500D
:100E9800FCEC51F0546E0A0E326E010E336E54C0E3
:100EA80034F0356A630E366E020EEEEC15F03250F1
:100EB800546E010E086E050E096E5450FCEC51F08C
:100EC800546E20EE01F05550D9265650DA2254C0FF
:100ED800DFFF7CEF08F0480E106EFB0E116EF7EC8A
:100EE80048F0010E086E630E096E5450FCEC51F088
:100EF800546E0E0E326E020E336E54C034F0356AE4
:100F0800630E366E020EEEEC15F03250546E010E82
:100F1800086E630E096E5450FCEC51F0546E20EECE
:100F280001F05550D9265650DA2254C0DFFF7CEF25
:100F380008F074C054F03F0E5464A5EF07F0A7EF13
:100F480007F0ABEF07F07CEF08F07CEF08F05450A7
:100F5800030D000EF324D96E030EF420DA6E000E92
:100F6800DF6E542A3F0E5464BCEF07F0BEEF07F063
:100F7800ABEF07F07CEF08F07CEF08F0E30E106EA3
:100F8800F60E116EF7EC48F00D0E326E050E336E4C
:100F980057C034F058C035F0030E366E020EEEEC32
:100FA80015F032C057F033C058F020EE01F055501C
:100FB800D9265650DA2257C0DFFF20EE02F05550EE
:100FC800D9265650DA225850DF6E7CEF08F0E30E2F
:100FD800106EF60E116EF7EC48F00D0E326E050E1F
:100FE800336E57C034F058C035F0030E366E020E1B
:100FF800EEEC15F032C057F033C058F020EE01F097
:101008005550D9265650DA2257C0DFFF20EE02F09D
:101018005550D9265650DA225850DF6E14EF08F092
:101028006C0E106EFC0E116EF7EC48F0010E086E97
:10103800050E096E5450FCEC51F0546E0E0E326ED3
:10104800010E336E54C034F0356A630E366E020EEC
:10105800EEEC15F03250546E010E086E050E096E56
:101068005450FCEC51F0546E20EE01F05550D92646
:101078005650DA2254C0DFFF7CEF08F07CEF08F00E
:101088000001C351000AD8B49DEF07F0040AD8B490
:101098006FEF07F0020AD8B4B3EF05F0010AD8B42D
:1010A800D1EF05F00F0AD8B40DEF06F0010AD8B455
:1010B8005AEF06F0030AD8B4A7EF06F0010AD8B42D
:1010C800EFEF05F0070AD8B441EF07F01D0AD8B4CE
:1010D800F4EF06F0040AD8B4C2EF07F0030AD8B454
:1010E800EBEF07F0010AD8B414EF08F07CEF08F032
:1010F80055C0D9FF56C0DAFFC3C0DFFF742A000EFF
:101108000001A16F0D0EA06FF2EC52F016EC2DF05D
:10111800D6EF08F0000E0001A16F0D0EA06FF2ECE3
:1011280052F016EC2DF0D6EF08F0D6EF08F0765016
:10113800300AD8B452EF05F0010AD8B452EF05F0DE
:10114800030AD8B452EF05F0010AD8B452EF05F0FB
:10115800070AD8B452EF05F0010AD8B452EF05F0E7
:10116800030AD8B452EF05F0010AD8B452EF05F0DB
:101178000F0AD8B452EF05F0010AD8B452EF05F0BF
:101188007A0AD8B48EEF08F00D0AD8B4F1EF04F05B
:10119800010AD8B49BEF05F01F0AD8B419EF05F07F
:1011A800D6EF08F07650D8B4DCEF08F0DEEF08F0A0
:1011B800E2EF08F076C0ABF0E2EF08F01200E2ECE4
:1011C80052F00001D86FC4EF0BF030EF0CF0000EB6
:1011D8000D6E030E93EC51F00D0E106EF90E116E9C
:1011E800F7EC48F030EF0CF0000E0D6E030E93ECA8
:1011F80051F0350E106EF90E116EF7EC48F030EF25
:101208000CF0000E0D6E030E93EC51F0210E106ED3
:10121800F90E116EF7EC48F030EF0CF082EC52F05A
:101228000001D66FD651640DF3CF4AF1F4CF4BF1DC
:10123800000E706E000E6F6E30EF0CF0000E0D6E2B
:10124800030E93EC51F00F0E106EF70E116EF7ECC3
:1012580048F030EF0CF01CEC50F008C0DEF009C08C
:10126800DFF0DEC0C6F0DFC0C7F00001C86BC96B95
:10127800B4C0CAF0CB6B8AEC24F030EF0CF01CEC55
:1012880050F008C0DEF009C0DFF00001B451D8B456
:1012980050EF09F052EF09F05AEF09F0DEC0D0F034
:1012A800DFC0D1F0ADEC52F030EF0CF0DEC0D0F082
:1012B800DFC0D1F0B7EC51F030EF0CF030EF0CF0AC
:1012C8001CEC50F008C0DEF009C0DFF00001DE5170
:1012D800DF11D8A472EF09F074EF09F07AEF09F082
:1012E800000EDF6F010EDE6F7AEF09F0100EDE5D83
:1012F800270EDF59D8A083EF09F085EF09F08BEFAF
:1013080009F0270EDF6F0F0EDE6F8BEF09F0DEC0DE
:101318009CF0DFC09DF0000E9B6F000E9A6F30EFBF
:101328000CF01CEC50F008C0DEF009C0DFF0000142
:101338009C519D11D8A4A3EF09F0A5EF09F0ADEFDA
:1013480009F0000E216E040E206E9DEC36F030EF91
:101358000CF0DEC0C6F0DFC0C7F00CEC2CF030EFAC
:101368000CF030EF0CF01CEC50F008C0DEF009C0B7
:10137800DFF000019C519D11D8A4C5EF09F0C7EF1B
:1013880009F0CFEF09F0000E216E040E206E9DECDF
:1013980036F030EF0CF00001B451D8B4D6EF09F0B4
:1013A800D8EF09F0E0EF09F0DE519A25DE6FDF5142
:1013B8009B21DF6F11EF0AF0DE519A5DDF519B59D7
:1013C800D8A0E9EF09F0EBEF09F0FBEF09F0DEC078
:1013D800D6F0DFC0D7F0D61FD71FD64BD72B9A51E0
:1013E800D625DE6F9B51D721DF6F11EF0AF0DEC0E3
:1013F800D6F0DFC0D7F0D61FD71FD64BD72B9A51C0
:10140800D6279B51D7239C51D625DE6F9D51D721D6
:10141800DF6F11EF0AF011EF0AF0DEC0C6F0DFC08F
:10142800C7F00CEC2CF030EF0CF030EF0CF082EC45
:1014380052F00001DD6FDD51D8A425EF0AF027EF47
:101448000AF02BEF0AF0010EDD6F2BEF0AF0050E04
:10145800DD6531EF0AF033EF0AF037EF0AF0050ED9
:10146800DD6F37EF0AF0FF0EDD259E6F9F6BFF0ED5
:101478009F2330EF0CF0010EB46F30EF0CF0000E2C
:10148800B46F30EF0CF0B451D8B44DEF0AF050EF10
:101498000AF0010E51EF0AF0000EB46F30EF0CF0B5
:1014A800070EAE655AEF0AF05CEF0AF064EF0AF037
:1014B800000E216E010E206E9DEC36F030EF0CF020
:1014C8000001AE51010D100EF324D96E010EF42067
:1014D800DA6E75C0DFFFAE51020D000EF324D96E2F
:1014E800010EF420DA6E000EDE6E000EDD6EAE2BFD
:1014F80030EF0CF030EF0CF0070EAE6586EF0AF017
:1015080088EF0AF090EF0AF0000E216E010E206EAF
:101518009DEC36F030EF0CF00001AE51010D100ECD
:10152800F324D96E010EF420DA6E75C0DFFF1CECCF
:1015380050F00001AE51020D000EF324D96E010ED9
:10154800F420DA6E08C0DEFF09C0DDFFAE2B30EFF5
:101558000CF030EF0CF0AE51D8A4B5EF0AF0B7EFAD
:101568000AF0BFEF0AF0000E216E020E206E9DEC0D
:1015780036F030EF0CF00001AE07AE51020D000E50
:10158800F324D96E010EF420DA6EDE50DE10D8B4E2
:10159800D0EF0AF0D2EF0AF0FDEF0AF0AE51020DDB
:1015A800000EF324D96E010EF420DA6EDE06000E6A
:1015B800DD5AAE51020D000EF324D96E010EF4204F
:1015C800DA6EDE50DE10D8B4ECEF0AF0EEEF0AF077
:1015D80030EF0CF0AE51010D100EF324D96E010E50
:1015E800F420DA6EDF50756EAE2B30EF0CF030EF72
:1015F8000CF0AE51010D100EF324D96E010EF4203B
:10160800DA6EDF50756EAE2B30EF0CF030EF0CF069
:1016180030EF0CF01CEC50F008C0DEF009C0DFF031
:10162800DEC021F0DFC022F0236A246A28EC4FF0E4
:1016380021C0D9F022C0DAF023C0DBF024C0DCF0EE
:10164800D9C065F0DAC066F0DBC067F0DCC068F0CE
:10165800C7EC40F030EF0CF09EC0AFF09EEC19F0F4
:1016680030EF0CF0809230EF0CF0000E0D6E030E90
:1016780093EC51F07B0E106EFC0E116EF7EC48F0F7
:101688001CEC50F008C0DEF009C0DFF0DEC0C6F088
:10169800DFC0C7F00001C86BC96B4EC1CAF04FC1AB
:1016A800CBF0B6EC3AF030EF0CF082EC52F00001DF
:1016B800DD6FDD51D8A463EF0BF065EF0BF069EF38
:1016C8000BF0010EDD6F69EF0BF0050EDD656FEFB6
:1016D8000BF071EF0BF075EF0BF0050EDD6F75EF8A
:1016E8000BF0FF0EDD2501014E6F4F6BFF0E4F23F0
:1016F80030EF0CF0000E0D6E030E93EC51F0970EC8
:10170800106EFE0E116EF7EC48F0000E0001C66F69
:10171800000EC76F000EC86F000EC96F000ECB6FAA
:10172800040ECA6FB6EC3AF030EF0CF01CEC50F037
:1017380008C0DEF009C0DFF0DEC021F0DFC022F013
:10174800236A246AF5EC4EF021C0D9F022C0DAF001
:1017580023C0DBF024C0DCF0D9C084F0DAC085F007
:10176800DBC086F0DCC087F030EF0CF0000E216E95
:10177800050E206E9DEC36F030EF0CF030EF0CF0DB
:101788000001D851000AD8B4BAEF0BF0010AD8B456
:10179800EBEF08F0030AD8B4F8EF08F0010AD8B460
:1017A80005EF09F0070AD8B412EF09F0010AD8B416
:1017B80022EF09F0030AD8B42FEF09F0010AD8B4D0
:1017C80043EF09F00F0AD8B464EF09F0010AD8B45E
:1017D80095EF09F0030AD8B4B7EF09F0010AD8B4B5
:1017E8000EEF0BF0070AD8B41BEF0AF0010AD8B4C1
:1017F8003FEF0AF0030AD8B443EF0AF0010AD8B45D
:1018080047EF0AF01F0AD8B454EF0AF0010AD8B417
:1018180080EF0AF0030AD8B4AFEF0AF0010AD8B48F
:1018280036EF0BF0070AD8B430EF0BF0010AD8B442
:1018380039EF0BF0030AD8B49AEF0BF0010AD8B4C9
:1018480059EF0BF00F0AD8B47EEF0BF0010AD8B4A9
:1018580030EF0CF030EF0CF01200B4EF0EF01BEC90
:1018680042F02AEC53F024EC46F00CEF0FF0080E8F
:10187800326E040E336E57C134F058C135F0FF0E86
:10188800366E010EEEEC15F032C057F133C058F148
:10189800050E326E040E336E5BC134F05CC135F058
:1018A800FF0E366E020EEEEC15F032C05BF133C05F
:1018B8005CF10E0E326E040E336E5DC134F05EC103
:1018C80035F0FF0E366E020EEEEC15F032C05DF10B
:1018D80033C05EF1070E326E020E336E59C134F01A
:1018E8005AC135F0010E366E030EEEEC15F032C01B
:1018F80059F133C05AF10101585107E10A0E575DF9
:10190800D8B089EF0CF08BEF0CF091EF0CF0000ED3
:10191800586F0A0E576F91EF0CF057515B5D585195
:101928005C59D8B09AEF0CF09CEF0CF0A2EF0CF0D9
:1019380057C15BF158C15CF1A2EF0CF05B515D5DE2
:101948005C515E59D8B0ABEF0CF0ADEF0CF0B3EFD3
:101958000CF05BC15DF15CC15EF1B3EF0CF02AECF9
:1019680053F00CEF0FF0010E326E060E336E6FC19E
:1019780034F070C135F071C136F072C137F0FF0E26
:10198800386E020EC9EC17F032C06FF133C070F137
:1019980034C071F135C072F16FC108F070C109F03F
:1019A80071C10AF072C10BF04EEC4EF0000E656E7C
:1019B800000E666E000E676E000E686E2AEC53F01D
:1019C8000CEF0FF001015F51D8B4EDEF0CF0F0EF20
:1019D8000CF0010EF1EF0CF0000E5F6F2AEC53F0E3
:1019E8000CEF0FF00C0E326E030E336E60C134F044
:1019F80061C135F0FF0E366E020EEEEC15F032C006
:101A080060F133C061F12AEC53F00CEF0FF00101E3
:101A18007351D8B412EF0DF015EF0DF0010E16EF5B
:101A28000DF0000E736F2AEC53F00CEF0FF001016C
:101A38007451D8B422EF0DF025EF0DF0010E26EF0A
:101A48000DF0000E746F2AEC53F00CEF0FF0010E3E
:101A5800326E020E336E75C134F076C135F0010E68
:101A6800366E020EEEEC15F032C075F133C076F129
:101A78000CEF0FF001017851D8B445EF0DF048EFA5
:101A88000DF0010E49EF0DF0000E786F2AEC53F0BF
:101A98000CEF0FF0BFAF53EF0DF055EF0DF059EF0E
:101AA8000DF069C0BFF05EEF0DF06950800FBF6F99
:101AB8005EEF0DF09BEC4CF00CEF0FF02AEC53F0BE
:101AC800010E04EC38F00CEF0FF0800E0001C01B83
:101AD800C0BF71EF0DF073EF0DF095EF0DF009EC4D
:101AE80000F0010E0D6E020E93EC51F0DD0E106E3B
:101AF800FE0E116EF7EC48F0050E0D6E020E93EC1B
:101B080051F0060E326E010E336E000E356E010E68
:101B1800346EFF0E366E020EEEEC15F032500001F8
:101B2800C06F9BEC4CF00CEF0FF0800E0101791B9D
:101B38002AEC53F00CEF0FF0800E01017A1B2AEC0F
:101B480053F00CEF0FF0080E326E040E336E7BC1AB
:101B580034F07CC135F0FF0E366E010EEEEC15F058
:101B680032C07BF133C07CF1050E326E040E336E49
:101B78007FC134F080C135F0FF0E366E020EEEECF8
:101B880015F032C07FF133C080F10E0E326E040EB4
:101B9800336E81C134F082C135F0FF0E366E020E0D
:101BA800EEEC15F032C081F133C082F1070E326ECF
:101BB800020E336E7DC134F07EC135F0010E366EF3
:101BC800030EEEEC15F032C07DF133C07EF1010159
:101BD8007C5107E10A0E7B5DD8B0F5EF0DF0F7EF09
:101BE8000DF0FDEF0DF0000E7C6F0A0E7B6FFDEF20
:101BF8000DF07B517F5D7C518059D8B006EF0EF017
:101C080008EF0EF00EEF0EF07BC17FF17CC180F182
:101C18000EEF0EF07F51815D80518259D8B017EFD9
:101C28000EF019EF0EF01FEF0EF07FC181F180C1A9
:101C380082F11FEF0EF02AEC53F00CEF0FF0090EB3
:101C4800326E040E336E83C134F084C135F0FF0E5A
:101C5800366E020EEEEC15F032C083F133C084F11B
:101C680001017F51835D80518459D8B03EEF0EF059
:101C780040EF0EF00CEF0FF07FC183F180C184F1CB
:101C88000CEF0FF00CEF0FF0010E326E050E336EF5
:101C98008AC134F08BC135F0FF0E366E020EEEECC1
:101CA80015F032C08AF133C08BF18AC124F18BC19F
:101CB80025F10101266B276B000E0001846F000ED1
:101CC800856F000E866F000E876F2AEC53F00CEFBD
:101CD8000FF001018651D8B474EF0EF077EF0EF0D3
:101CE800010E78EF0EF0000E866F2AEC53F00CEF21
:101CF8000FF001018551D8B484EF0EF087EF0EF094
:101D0800010E88EF0EF0000E856F2AEC53F00CEFF1
:101D18000FF0010E326E040E336E8CC134F08DC19B
:101D280035F0020E366E020EEEEC15F032C08CF174
:101D380033C08DF12AEC53F00CEF0FF001018751FD
:101D4800D8B4A9EF0EF0ACEF0EF0010EADEF0EF027
:101D5800000E876F2AEC53F00CEF0FF00CEF0FF02A
:101D68000001A651000AD8B43BEF0CF0010AD8B420
:101D7800B7EF0CF0030AD8B4E6EF0CF0010AD8B4B8
:101D8800F6EF0CF0070AD8B40BEF0DF0010AD8B43F
:101D98001BEF0DF0030AD8B42BEF0DF0010AD8B4ED
:101DA8004EEF0DF00F0AD8B462EF0DF0010AD8B467
:101DB80069EF0DF0030AD8B433EF0CF0010AD8B478
:101DC80099EF0DF0070AD8B4A0EF0DF0010AD8B4C6
:101DD800A7EF0DF0030AD8B423EF0EF0010AD8B428
:101DE80048EF0EF01F0AD8B46DEF0EF0010AD8B410
:101DF8007DEF0EF0030AD8B48DEF0EF0010AD8B4C7
:101E0800A2EF0EF0070AD8B43EEF0DF00CEF0FF07A
:101E1800120020EE02F02350D9262450DA22DF5097
:101E2800276E2750296E286A20EE01F02350D92604
:101E38002450DA22DF502A6E2A5028242C6E000EF5
:101E480029202D6E20EE01F02350D9262450DA22C5
:101E5800DF502B6E000E0D6E1F5093EC51F02128B1
:101E680016EC53F0200E05EC4BF0040E0D6E1F50CF
:101E780093EC51F05DEF11F02550D8B446EF0FF018
:101E880048EF0FF050EF0FF09F0E106EFA0E116E24
:101E9800F7EC48F0CCEF11F0ED0E106EFF0E116E5E
:101EA800F7EC48F0CCEF11F0CCEF11F0210E106EEA
:101EB800FE0E116EF7EC48F0CCEF11F0A80E106E84
:101EC800FC0E116EF7EC48F0CCEF11F02F0E106EEF
:101ED800FC0E116EF7EC48F0CCEF11F0160E106EF8
:101EE800FE0E116EF7EC48F02650D8B47EEF0FF0D6
:101EF80080EF0FF08BEF0FF02BC015F0166A020E73
:101F0800176E010E186EAAEC41F0CCEF11F0740EAA
:101F1800106EFF0E116EF7EC48F0CCEF11F0CCEF1D
:101F280011F0280E106EFD0E116EF7EC48F0CCEF94
:101F380011F06D0E106EFF0E116EF7EC48F0265082
:101F4800D8B4A9EF0FF0ABEF0FF0B3EF0FF02CC040
:101F58001BF02DC01CF0D5EC4DF0CCEF11F0050EA8
:101F6800106EFF0E116EF7EC48F0CCEF11F0CCEFCD
:101F780011F0BB0E106EFE0E116EF7EC48F02650F5
:101F8800D8B4C9EF0FF0CBEF0FF0D3EF0FF02CC0A0
:101F98001BF02DC01CF0D5EC4DF0CCEF11F0050E68
:101FA800106EFF0E116EF7EC48F0CCEF11F0CCEF8D
:101FB80011F0690E106EFE0E116EF7EC48F0265007
:101FC800D8B4E9EF0FF0EBEF0FF0F7EF0FF02CC0FC
:101FD80015F02DC016F0040E176E010E186EAAEC3F
:101FE80041F0CCEF11F0E90E106EFF0E116EF7EC18
:101FF80048F0CCEF11F0CCEF11F0550E106EFE0E3C
:10200800116EF7EC48F02650D8B40DEF10F00FEF32
:1020180010F01BEF10F02CC015F02DC016F0040EB8
:10202800176E010E186EAAEC41F0CCEF11F0E90E14
:10203800106EFF0E116EF7EC48F0CCEF11F0CCEFFC
:1020480011F0A00E106EFE0E116EF7EC48F026503F
:10205800D8B431EF10F033EF10F03FEF10F02CC090
:1020680015F02DC016F0040E176E010E186EAAECAE
:1020780041F0CCEF11F0E90E106EFF0E116EF7EC87
:1020880048F0CCEF11F0CCEF11F00F0E106EFE0EF1
:10209800116EF7EC48F02650D8B455EF10F057EF12
:1020A80010F062EF10F02BC015F0166A010E176ED3
:1020B800000E186EAAEC41F0CCEF11F0E90E106E8C
:1020C800FF0E116EF7EC48F0CCEF11F0CCEF11F0E9
:1020D8005D0E106EFD0E116EF7EC48F0CCEF11F0AE
:1020E8001A0E106EFD0E116EF7EC48F0CCEF11F0E1
:1020F800990E106EFC0E116EF7EC48F0CCEF11F053
:102108006A0E106EFD0E116EF7EC48F0CCEF11F070
:102118005F0E106EFE0E116EF7EC48F02650D8B424
:1021280098EF10F09AEF10F0A6EF10F02CC015F011
:102138002DC016F0030E176E010E186EAAEC41F0B2
:10214800CCEF11F00D0E106EFF0E116EF7EC48F08B
:10215800CCEF11F0CCEF11F0C40E106EFE0E116E24
:10216800F7EC48F0CCEF11F0A90E106EFE0E116ED0
:10217800F7EC48F02650D8B4C4EF10F0C6EF10F0D2
:10218800CEEF10F02CC01BF02DC01CF0D5EC4DF09C
:10219800CCEF11F0050E106EFF0E116EF7EC48F043
:1021A800CCEF11F0CCEF11F02C0E106EFE0E116E6C
:1021B800F7EC48F0CCEF11F0A70E106EFD0E116E83
:1021C800F7EC48F0CCEF11F0F10E106EFF0E116E27
:1021D800F7EC48F0CCEF11F04B0E106EFE0E116EBE
:1021E800F7EC48F02650D8B4FCEF10F0FEEF10F0F2
:1021F80006EF11F02CC01BF02DC01CF0D5EC4DF0F3
:10220800CCEF11F0DC0E106EFF0E116EF7EC48F0FB
:10221800CCEF11F0CCEF11F0250E106EFF0E116E01
:10222800F7EC48F0CCEF11F0B20E106EFE0E116E06
:10223800F7EC48F02650D8B424EF11F026EF11F04F
:102248002EEF11F02CC01BF02DC01CF0D5EC4DF07A
:10225800CCEF11F0DC0E106EFF0E116EF7EC48F0AB
:10226800CCEF11F0CCEF11F00B0E106EFE0E116ECC
:10227800F7EC48F02650D8B444EF11F046EF11F0CF
:1022880051EF11F02BC015F0166A010E176E000EF3
:10229800186EAAEC41F0CCEF11F0E90E106EFF0EAB
:1022A800116EF7EC48F0CCEF11F0CCEF11F0CCEF59
:1022B80011F023C0D9FF24C0DAFFDF50000AD8B4D8
:1022C80040EF0FF0010AD8B45AEF0FF0030AD8B460
:1022D80062EF0FF0010AD8B46AEF0FF0070AD8B41A
:1022E80072EF0FF0010AD8B495EF0FF0030AD8B4D3
:1022F8009DEF0FF0010AD8B4BDEF0FF00F0AD8B464
:10230800DDEF0FF0010AD8B401EF10F0030AD8B4DA
:1023180025EF10F0010AD8B4B8EF10F0070AD8B4C6
:1023280049EF10F0010AD8B46CEF10F0030AD8B4E2
:1023380074EF10F0010AD8B47CEF10F01F0AD8B47B
:1023480084EF10F0010AD8B48CEF10F0030AD8B467
:10235800B0EF10F0010AD8B4E0EF10F0070AD8B4D3
:10236800D8EF10F0010AD8B4F0EF10F0030AD8B48F
:1023780018EF11F0010AD8B438EF11F00F0AD8B4E9
:1023880010EF11F0010AD8B4E8EF10F0CCEF11F01B
:10239800490E106EFE0E116EF7EC48F01200E2ECDA
:1023A80052F0646E0001B251D8A4DDEF11F0DFEFF6
:1023B80011F0E3EF11F0E3EC08F0E3EF11F0010E98
:1023C8000001B26FBAEF13F0A2EC50F00009D8A4E4
:1023D800F0EF11F0F2EF11F0FDEF11F00001B15143
:1023E800D8B4F9EF11F0FBEF11F0F1EF13F0FDEFB6
:1023F80011F0FFEC52F09EEC19F0F1EF13F0F1EF51
:1024080013F0DAEC51F00009D8A40DEF12F00FEF39
:1024180012F01AEF12F00001B151D8B416EF12F011
:1024280018EF12F0F1EF13F01AEF12F0FFEC52F080
:102438009EEC19F0F1EF13F0F1EF13F0DAEC51F034
:102448000009D8B42AEF12F02CEF12F037EF12F08F
:102458000001B151D8B433EF12F035EF12F0F1EFBB
:1024680013F037EF12F0FFEC52F09EEC19F0F1EF99
:1024780013F0F1EF13F0000E0D6E030E93EC51F014
:102488009B0E106EFD0E116EF7EC48F06FC0E0F079
:1024980070C0E1F00001E01FE11FE04BE12B0101FA
:1024A8004A510001E02701014B510001E123630E6D
:1024B800E025086E000EE121096E000E0B6E640E19
:1024C8000A6E91EC4BF008C015F009C016F0020E28
:1024D800176E010E186EAAEC41F06F5001014A5DAB
:1024E80070504B59D8A07BEF12F07DEF12F088EFB7
:1024F80012F00001B151D8B484EF12F086EF12F057
:10250800F1EF13F088EF12F0FFEC52F0F1EF13F057
:10251800F1EF13F04F0E7618D8B495EF12F097EF4D
:1025280012F0A2EF12F00001B151D8B49EEF12F0F0
:10253800A0EF12F0F1EF13F0A2EF12F0FFEC52F05F
:102548009EEC19F0F1EF13F0F1EF13F0ACEF12F08D
:10255800000E106E140E116E020E1EEC51F00001EA
:10256800EE51EF11D8B4BBEF12F0BDEF12F0F1EF5E
:1025780013F0FFEC52F0F1EF13F0F1EF13F0C7EFA7
:1025880012F0C7EF12F09AC01BF09BC01CF09CC061
:102598001DF09DC01EF048EC48F00001EE51EF110F
:1025A800D8B4D9EF12F0DBEF12F0F1EF13F0FFEC33
:1025B80052F0F1EF13F0F1EF13F0E3EF12F084C0F3
:1025C80022F085C023F086C024F087C025F0000ED5
:1025D800276E010E266E000E296E020E286EF4EC90
:1025E8003BF00001EE51EF11D8B4FDEF12F0FFEF10
:1025F80012F0F1EF13F0FFEC52F0F1EF13F0F1EFFE
:1026080013F0050E0D6E000E93EC51F0AB0E106E2C
:10261800FF0E116EF7EC48F0000E0D6E030E93ECF2
:1026280051F05D0E106EF90E116EF7EC48F087EF61
:1026380013F0000E0001D16F010ED06FADEC52F017
:10264800F1EF13F0000E0001D16F010ED06FB7EC5F
:1026580051F0F1EF13F0000E0001D16F0A0ED06FA8
:10266800ADEC52F0F1EF13F0000E0001D16F0A0E3D
:10267800D06FB7EC51F0F1EF13F0000E0001D16FFD
:10268800640ED06FADEC52F0F1EF13F0000E0001C4
:10269800D16F640ED06FB7EC51F0F1EF13F0030E69
:1026A8000001D16FE80ED06FADEC52F0F1EF13F0EE
:1026B800030E0001D16FE80ED06FB7EC51F0F1EFC7
:1026C80013F0000E1F6E000E1E6E6DEC51F0F1EF50
:1026D80013F0050E106E050E116E000E1EEC51F073
:1026E800000E106E140E116E030E1EEC51F0AFC0EA
:1026F8009EF000019F6B9EEC19F0FFEC52F0F1EF99
:1027080013F0F1EF13F07650310AD8B426EF13F036
:10271800020AD8B41DEF13F0070AD8B438EF13F043
:10272800020AD8B42FEF13F0010AD8B44AEF13F015
:102738000E0AD8B441EF13F0770AD8B453EF13F068
:10274800010AD8B46DEF13F01F0AD8B45CEF13F088
:10275800030AD8B465EF13F0F1EF13F0F1EF13F0BB
:10276800FFEC52F0F1EF13F0F1EF13F06450010AAF
:10277800D8B4E8EF11F0030AD8B405EF12F0010A53
:10278800D8B422EF12F0070AD8B43FEF12F0010ACA
:10279800D8B48EEF12F0030AD8B4ACEF12F0010AE5
:1027A800D8B4ACEF12F00F0AD8B4C7EF12F0010A90
:1027B800D8B4C7EF12F0030AD8B4C7EF12F01E0A54
:1027C800D8B405EF13F0010AD8B4E3EF12F00D0AFC
:1027D800D8B4E3EF12F0B4EF13F012009AEF15F04B
:1027E8005FEF14F0000E0001A16F010EA06FEDEF76
:1027F80015F0000E0001A16F030EA06FEDEF15F0AC
:10280800000E0001A16F070EA06FEDEF15F0000E8E
:102818000001A16F090EA06FEDEF15F001017A51CB
:10282800D8B419EF14F01BEF14F0EDEF15F0000E0B
:102838000001A16F050EA06FEDEF15F0EDEF15F09B
:1028480001017951D8B42BEF14F02DEF14F0EDEF0E
:1028580015F0000E0001A16F0B0EA06FEDEF15F043
:10286800EDEF15F0000E0001A16F0F0EA06FEDEF58
:1028780015F0960E176E430E8DEC4FF00009D8B484
:1028880048EF14F04AEF14F0EDEF15F0000E096E62
:10289800FA0E086E000E0B6E320E0A6EE8EC49F066
:1028A800000E04EC38F024EC46F0EDEF15F0EDEFF7
:1028B80015F0EDEF15F07650310AD8B4F6EF13F0B5
:1028C800030AD8B4FDEF13F0010AD8B404EF14F0EA
:1028D800070AD8B40BEF14F0010AD8B412EF14F0B9
:1028E8000D0AD8B424EF14F0010AD8B436EF14F066
:1028F8007A0AD8B43DEF14F0EDEF15F0EDEF15F0CE
:10290800F2EC52F0D70E106EFF0E116EF7EC48F095
:10291800C7EC40F0000E1C6E000E1B6E18EC4CF05D
:10292800000E0001A16F020EA06FEDEF15F028EC6C
:102938001DF0EDEF15F046EC51F06D506E10D8B467
:10294800A8EF14F0AAEF14F0AEEF14F024EC46F060
:10295800EDEF15F0000E6C6E000E6B6E000E656EDE
:10296800000E666E000E676E000E686E000E0001A7
:10297800806F000E816F000E826F000E836F1DEC5A
:1029880052F0000E1C6E010E1B6E18EC4CF0000E7F
:102998000001A16F040EA06FEDEF15F0EDEF15F03B
:1029A800BAEC21F0EDEF15F0C6EC29F06D506E1081
:1029B800D8B4E1EF14F0E3EF14F0E7EF14F024ECEF
:1029C80046F0EDEF15F0000E6C6E000E6B6E000E0B
:1029D800656E000E666E000E676E000E686E1AEC6D
:1029E8004DF0000E1C6E010E1B6E18EC4CF0CCEC7A
:1029F80050F0000E0001A16F060EA06FEDEF15F06C
:102A0800EDEF15F03EEC47F0EDEF15F098EC47F0E0
:102A18006D506E10D8B413EF15F015EF15F019EFCF
:102A280015F024EC46F0EDEF15F06CEC52F0000ECA
:102A38001C6E020E1B6E18EC4CF0000E0001A16F0C
:102A4800080EA06FEDEF15F0EDEF15F06CEC1BF034
:102A5800EDEF15F0F2EC52F08F0E106EFD0E116EC8
:102A6800F7EC48F0000E0D6E030E93EC51F0EF0EEC
:102A7800106EFB0E116EF7EC48F0C7EC40F0000E3C
:102A88001C6E030E1B6E18EC4CF0000E0001A16FBB
:102A98000A0EA06FEDEF15F0E4EC35F0EDEF15F050
:102AA800F2EC52F08E0E106EFE0E116EF7EC48F03E
:102AB800000E0D6E010E93EC51F06A0E106EFA0EB8
:102AC800116EF7EC48F0000E0D6E020E93EC51F00B
:102AD800360E106EFB0E116EF7EC48F0000E0D6E00
:102AE800030E93EC51F0570E106EFA0E116EF7ECC0
:102AF80048F0000E0001A16F0C0EA06FEDEF15F06D
:102B08009FEC49F0EDEF15F0F9EC42F0EDEF15F020
:102B1800C6EC04F0EDEF15F055EC52F0EDEF15F0C2
:102B280096EC33F0EDEF15F0EDEF15F0A0C0E8F0FE
:102B3800A1C0E9F00001E951000AD8B4A6EF15F0E8
:102B4800EDEF15F0E851000AD8B45FEF14F0010A70
:102B5800D8B484EF14F0030AD8B49BEF14F0010A38
:102B6800D8B49FEF14F0070AD8B4D4EF14F0010AD0
:102B7800D8B4D8EF14F0030AD8B406EF15F0010A58
:102B8800D8B40AEF15F00F0AD8B42AEF15F0010AE5
:102B9800D8B42EEF15F0030AD8B450EF15F0010A97
:102BA800D8B454EF15F0070AD8B484EF15F0010A29
:102BB800D8B488EF15F0030AD8B48CEF15F0010AE1
:102BC800D8B490EF15F01F0AD8B494EF15F0EDEFD4
:102BD80015F012004B6E34C046F035C047F0486A15
:102BE800496A000E456E010E446E000E6E6E000EB0
:102BF8006D6E32C021F033C022F034C023F035C0EE
:102C080024F0256A266A36C027F03E0E286E000E8C
:102C1800296E4B5061EC39F0000E4C6E32040D6E8B
:102C28004B5093EC51F05B0E05EC4BF03350365C97
:102C3800D8A021EF16F024EF16F0010E25EF16F0BC
:102C4800000E4A6E325033244A240D6E4B5093ECDA
:102C580051F05D0E05EC4BF032C00DF04B5093EC8B
:102C680051F081900F0ED5EC4BF081900E0ED5EC03
:102C78004BF071EF17F09EEC19F034EF17F055EFA9
:102C880016F055EF16F055EF16F055EF16F055EF14
:102C980016F055EF16F055EF16F055EF16F055EF04
:102CA80016F04C50010D3E0EF324D96E000EF420A0
:102CB800DA6E76C0DFFF4C50010D3E0EF324D96E5C
:102CC800000EF420DA6EDF5005EC4BF06CEF16F0D6
:102CD800FF0E376EFF0E386E3350396E3A6A375032
:102CE800392638503A224C503B6E3C6A39503B5C8E
:102CF8003C50800A3D6E3A50800A3D58D8B087EF64
:102D080016F089EF16F08CEF16F04C2A8CEF16F0BF
:102D180036504C5CD8B093EF16F096EF16F0010ED3
:102D280097EF16F0000E4A6E32504C244A240D6E6E
:102D38004B5093EC51F071EF17F04C50D8B4A7EF0B
:102D480016F0A9EF16F0ACEF16F04C06ACEF16F043
:102D580036504C5CD8B0B3EF16F0B6EF16F0010E53
:102D6800B7EF16F0000E4A6E32504C244A240D6E0E
:102D78004B5093EC51F071EF17F0000E456E000EBA
:102D8800446E000E6E6E010E6D6E71EF17F0000E40
:102D98004C6E000E466E000E476E000E486E000E1A
:102DA800496E0FEF17F046C008F047C009F048C059
:102DB8000AF049C00BF00A0E0C6E000E0D6E000EE4
:102DC8000E6E000E0F6E87EC4EF008C046F009C07C
:102DD80047F00AC048F00BC049F0D00E376EFF0E1E
:102DE800386E4C50010D3E0EF324D96E000EF420BF
:102DF800DA6EDF50396E3A6A3750392638503A223F
:102E0800395046263A504722000E4822000E4922E1
:102E18004C2A0FEF17F033504C5CD8A016EF17F080
:102E280018EF17F0D7EF16F01AEF17F0495008E12E
:102E38004804D8A022EF17F024EF17F02CEF17F072
:102E4800FF0E466EFF0E476E000E486E000E496E6E
:102E5800000E456E000E446E71EF17F071EF17F01B
:102E68007650300AD8B455EF16F0010AD8B455EFA9
:102E780016F0030AD8B455EF16F0010AD8B455EF86
:102E880016F0070AD8B455EF16F0010AD8B455EF72
:102E980016F0030AD8B455EF16F0010AD8B455EF66
:102EA80016F00F0AD8B455EF16F0010AD8B455EF4A
:102EB80016F07A0AD8B4C1EF16F00D0AD8B46CEF40
:102EC80016F0010AD8B4CBEF16F01F0AD8B4A1EF58
:102ED80016F071EF17F071EF17F044504510D8A4B1
:102EE80078EF17F07AEF17F03FEF16F07CEF17F056
:102EF8006D506E10D8B483EF17F085EF17F0A0EF80
:102F080017F032C021F033C022F034C023F035C0AE
:102F180024F0256A266A36C027F03E0E286E000E79
:102F2800296E4B5061EC39F034C046F035C047F09B
:102F3800486A496AA0EF17F081900C0ED5EC4BF067
:102F480032040D6E4B5093EC51F0200E05EC4BF013
:102F58003350365CD8A0B3EF17F0B6EF17F0010E78
:102F6800B7EF17F0000E4A6E325033244A240D6E24
:102F78004B5093EC51F0200E05EC4BF046C032F06C
:102F880047C033F0C8EF17F012004F6E34C04AF054
:102F980035C04BF036C04CF037C04DF0000E496ECE
:102FA800010E486E000E6E6E000E6D6E32C021F07E
:102FB80033C022F034C023F035C024F036C025F0E9
:102FC80037C026F038C027F0400E286E000E296E54
:102FD8004F5061EC39F0000E506E32040D6E4F50B8
:102FE80093EC51F05B0E05EC4BF03350385CD8A0F5
:102FF80000EF18F003EF18F0010E04EF18F0000EC0
:103008004E6E325033244E240D6E4F5093EC51F0D7
:103018005D0E05EC4BF032C00DF04F5093EC51F0C3
:1030280081900F0ED5EC4BF081900E0ED5EC4BF045
:103038003EEF19F09EEC19F001EF19F034EF18F09B
:1030480034EF18F034EF18F034EF18F034EF18F0CC
:1030580034EF18F034EF18F034EF18F034EF18F0BC
:103068005050010D400EF324D96E000EF420DA6E94
:1030780076C0DFFF5050010D400EF324D96E000ECC
:10308800F420DA6EDF5005EC4BF04BEF18F0FF0E32
:10309800396EFF0E3A6E33503B6E3C6A39503B2610
:1030A8003A503C2250503D6E3E6A3B503D5C3E508B
:1030B800800A3F6E3C50800A3F58D8B066EF18F03F
:1030C80068EF18F06BEF18F0502A6BEF18F03850D3
:1030D800505CD8B072EF18F075EF18F0010E76EF6B
:1030E80018F0000E4E6E325050244E240D6E4F5084
:1030F80093EC51F03EEF19F05050D8B486EF18F029
:1031080088EF18F08BEF18F050068BEF18F0385056
:10311800505CD8B092EF18F095EF18F0010E96EFCA
:1031280018F0000E4E6E325050244E240D6E4F5043
:1031380093EC51F03EEF19F0000E496E000E486E08
:10314800000E6E6E010E6D6E3EEF19F0000E506EA1
:10315800000E4A6E000E4B6E000E4C6E000E4D6E49
:10316800EEEF18F04AC008F04BC009F04CC00AF066
:103178004DC00BF00A0E0C6E000E0D6E000E0E6E9A
:10318800000E0F6E87EC4EF008C04AF009C04BF0F5
:103198000AC04CF00BC04DF0D00E396EFF0E3A6EDF
:1031A8005050010D400EF324D96E000EF420DA6E53
:1031B800DF503B6E3C6A39503B263A503C223B502C
:1031C8004A263C504B22000E4C22000E4D22502A1B
:1031D800EEEF18F03350505CD8A0F5EF18F0F7EF89
:1031E80018F0B6EF18F0F9EF18F0000E496E000E5F
:1031F800486E3EEF19F03EEF19F07650300AD8B419
:1032080034EF18F0010AD8B434EF18F0030AD8B430
:1032180034EF18F0010AD8B434EF18F0070AD8B41C
:1032280034EF18F0010AD8B434EF18F0030AD8B410
:1032380034EF18F0010AD8B434EF18F00F0AD8B4F4
:1032480034EF18F0010AD8B434EF18F07A0AD8B479
:10325800A0EF18F00D0AD8B44BEF18F0010AD8B453
:10326800AAEF18F01F0AD8B480EF18F03EEF19F053
:103278003EEF19F048504910D8A445EF19F047EF30
:1032880019F01EEF18F049EF19F06D506E10D8B410
:1032980050EF19F052EF19F071EF19F032C021F028
:1032A80033C022F034C023F035C024F036C025F0F6
:1032B80037C026F038C027F0400E286E000E296E61
:1032C8004F5061EC39F034C04AF035C04BF036C08D
:1032D8004CF037C04DF071EF19F081900C0ED5EC21
:1032E8004BF032040D6E4F5093EC51F0200E05EC6C
:1032F8004BF03350385CD8A084EF19F087EF19F001
:10330800010E88EF19F0000E4E6E325033244E2411
:103318000D6E4F5093EC51F0200E05EC4BF04AC067
:1033280032F04BC033F04CC034F04DC035F09DEF57
:1033380019F01200D80E156E010E166E080E000157
:10334800C161A9EF19F0ABEF19F0B9EF19F0C1514C
:10335800020D8E0EF324D96E010EF420DA6EDECF44
:1033680015F0DDCF16F0B9EF19F0000E776E8380F7
:10337800839283948396320E116ECAEF19F000F08F
:1033880000F000F000F000F000F000F0112EC3EFA4
:1033980019F083A8D2EF19F0D4EF19F0DCEF19F087
:1033A80015C0D9FF16C0DAFFDF50776EDCEF19F0D1
:1033B80083AAE1EF19F0E3EF19F0EDEF19F020EE31
:1033C80001F01550D9261650DA22DF50776EEDEF4E
:1033D80019F083ACF2EF19F0F4EF19F0FEEF19F0E1
:1033E80020EE02F01550D9261650DA22DF50776EFB
:1033F800FEEF19F083AE03EF1AF005EF1AF00FEFA6
:103408001AF020EE03F01550D9261650DA22DF50B4
:10341800776E0FEF1AF083908382320E126E1CEFD4
:103428001AF000F000F000F000F000F000F000F0FA
:10343800122E15EF1AF083A824EF1AF026EF1AF0CF
:1034480030EF1AF020EE04F01550D9261650DA2283
:10345800DF50776E30EF1AF083AA35EF1AF037EFA6
:103468001AF041EF1AF020EE05F01550D926165043
:10347800DA22DF50776E41EF1AF083AC46EF1AF08C
:1034880048EF1AF052EF1AF020EE06F01550D92640
:103498001650DA22DF50776E52EF1AF083AE57EFEC
:1034A8001AF059EF1AF063EF1AF020EE07F01550F2
:1034B800D9261650DA22DF50776E63EF1AF083921E
:1034C8008384320E136E70EF1AF000F000F000F0F3
:1034D80000F000F000F000F0132E69EF1AF083A856
:1034E80078EF1AF07AEF1AF084EF1AF020EE08F06D
:1034F8001550D9261650DA22DF50776E84EF1AF06D
:1035080083AA89EF1AF08BEF1AF095EF1AF020EEE4
:1035180009F01550D9261650DA22DF50776E95EF4C
:103528001AF083AC9AEF1AF09CEF1AF0A6EF1AF093
:1035380020EE0AF01550D9261650DA22DF50776EA1
:10354800A6EF1AF083AEABEF1AF0ADEF1AF0B7EFB3
:103558001AF020EE0BF01550D9261650DA22DF505B
:10356800776EB7EF1AF083948386320E146EC4EF29
:103578001AF000F000F000F000F000F000F000F0A9
:10358800142EBDEF1AF083A8CCEF1AF0CEEF1AF084
:10359800D8EF1AF020EE0CF01550D9261650DA2282
:1035A800DF50776ED8EF1AF083AADDEF1AF0DFEF5D
:1035B8001AF0E9EF1AF020EE0DF01550D926165042
:1035C800DA22DF50776EE9EF1AF083ACEEEF1AF0EB
:1035D800F0EF1AF0FAEF1AF020EE0EF01550D92697
:1035E8001650DA22DF50776EFAEF1AF083AEFFEF4B
:1035F8001AF001EF1BF00BEF1BF020EE0FF0155047
:10360800D9261650DA22DF50776E0BEF1BF080A018
:1036180010EF1BF012EF1BF02EEF1BF00001BA5158
:10362800D8A419EF1BF01BEF1BF02EEF1BF00A0EAE
:103638005BEC4FF080A023EF1BF025EF1BF02EEF83
:103648001BF0010E0001BA6F2EEF1BF02EEF1BF0DE
:103658002EEF1BF00001BB517718D8B436EF1BF0E2
:1036680038EF1BF064EF1BF07750D8B43EEF1BF037
:1036780040EF1BF050EF1BF0000E096EFA0E086EBB
:10368800000E0B6E320E0A6EE8EC49F077C0BBF004
:1036980077C076F068EF1BF00001B92B130EB965FF
:1036A80058EF1BF05AEF1BF068EF1BF077C0BBF028
:1036B80077C076F068EF1BF068EF1BF068EF1BF03F
:1036C800000E766E000EB96F77506BEF1BF012008C
:1036D8007650D8A472EF1BF074EF1BF00CEF1DF0BE
:1036E800A2EC50F00009D8B47CEF1BF07EEF1BF081
:1036F8000CEF1DF04E0E766E0CEF1DF00CEF1DF06A
:103708000CEF1DF06BC1D0F06CC1D1F06DC1D2F0DF
:103718006EC1D3F00001D01FD11FD21FD31FD02BF1
:10372800000ED123D223D3238051D025DE6F8151BF
:10373800D121DF6F8251D221E06F8351D321E16F14
:10374800A751D8B4AAEF1BF0ACEF1BF0CDEF1BF0DC
:103758001CC1DEF01DC1DFF01EC1E0F01FC1E1F0A9
:10376800010144514511D8B4BCEF1BF0BEEF1BF06A
:10377800CDEF1BF021EE6BF0DE500001DE5FDE5076
:10378800DF5BDE50E05BDD50E15BCDEF1BF0CDEFA2
:103798001BF0DEC0C6F0DFC0C7F0E0C0C8F0E1C073
:1037A800C9F0000E0001CB6F000ECA6F8AEC24F03E
:1037B80027EF1DF00001805101016B250001DE6F2C
:1037C800815101016C210001DF6F825101016D21DE
:1037D8000001E06F835101016E210001E16FA751E3
:1037E800D8B4F9EF1BF0FBEF1BF01CEF1CF01CC169
:1037F800DEF01DC1DFF01EC1E0F01FC1E1F00101E4
:1038080044054511D8B40BEF1CF00DEF1CF01CEF6C
:103818001CF021EE6BF0DE500001DE27DE50DF23C6
:10382800DE50E023DD50E1231CEF1CF01CEF1CF000
:10383800DEC0C6F0DFC0C7F0E0C0C8F0E1C0C9F024
:10384800000E0001CB6F010ECA6F8AEC24F027EF3F
:103858001DF0000E1F6E020E1E6E6DEC51F027EF6C
:103868001DF0070E326E050E336E80C034F081C035
:1038780035F0030E366E010EEEEC15F032C0DEF0B8
:1038880033C0DFF00001E06BE16B6D506E10D8A41F
:1038980050EF1CF052EF1CF027EF1DF080C0D0F065
:1038A80081C0D1F082C0D2F083C0D3F0D01FD11F25
:1038B800D21FD31FD02B000ED123D223D323DE5106
:1038C800D025D46FDF51D121D56FE051D221D66FE9
:1038D800E151D321D76FA00ED425DA6F8C0ED521F4
:1038E800DB6F000ED621DC6F000ED721DD6FDDBF48
:1038F8008AEF1CF0DD51DC110BE1A10EDA5D8C0EB4
:10390800DB59D8A08AEF1CF08CEF1CF094EF1CF068
:10391800600EDA27730EDB23FF0EDC23FF0EDD2398
:10392800DDBFA3EF1CF0DD51DC110BE1510EDA5DB8
:10393800460EDB59D8A0A3EF1CF0A5EF1CF0ABEFA7
:103948001CF0000ED96F000ED86FB1EF1CF0000EFE
:10395800D96F010ED86FB1EF1CF0E1BFC2EF1CF0B8
:10396800E151E01109E1A00EDE5D8C0EDF59D8B0FF
:10397800C0EF1CF0C2EF1CF0DFEF1CF0D8C018F04D
:10398800D9C019F032EC44F018501910D8B4CFEF60
:103998001CF0D1EF1CF0DFEF1CF0DEC0C6F0DFC07A
:1039A800C7F0E0C0C8F0E1C0C9F098C0CAF099C03B
:1039B800CBF08AEC24F06CEC52F027EF1DF027EFE7
:1039C8001DF024EC46F027EF1DF097EC4DF00009B0
:1039D800D8B4F1EF1CF0F3EF1CF027EF1DF0000E48
:1039E800656E000E666E000E676E000E686E000E45
:1039F8000001806F000E816F000E826F000E836FD2
:103A08006CEC52F027EF1DF027EF1DF027EF1DF0AB
:103A18007650300AD8B4E9EF1CF0730AD8B4E5EF51
:103A28001CF00D0AD8B4DEEF1BF0010AD8B435EF4C
:103A38001CF01F0AD8B486EF1BF0030AD8B42DEF88
:103A48001CF027EF1DF012007DEF1EF0000E0001A4
:103A5800D16F010ED06FADEC52F0B0EF1EF0000E3A
:103A68000001D16F010ED06FB7EC51F0B0EF1EF02E
:103A7800000E0001D16F0A0ED06FADEC52F0B0EF1E
:103A88001EF0000E0001D16F0A0ED06FB7EC51F096
:103A9800B0EF1EF0000E0001D16F640ED06FADECD8
:103AA80052F0B0EF1EF0000E0001D16F640ED06F1F
:103AB800B7EC51F0B0EF1EF0030E0001D16FE80E25
:103AC800D06FADEC52F0B0EF1EF0030E0001D16FD5
:103AD800E80ED06FB7EC51F0B0EF1EF0000E1F6E7D
:103AE800000E1E6E6DEC51F0B0EF1EF024EC46F0A7
:103AF800B0EF1EF065C008F066C009F067C00AF0B4
:103B080068C00BF0A00E0C6E8C0E0D6E000E0E6EC3
:103B1800000E0F6E87EC4EF008C014F009C015F0C7
:103B28000AC016F00BC017F088C018F089C019F049
:103B38008AC01AF08BC01BF02EEC3DF014C080F048
:103B480015C081F016C082F017C083F0050E326EE2
:103B5800050E336E80C034F081C035F0030E366E2A
:103B6800010EEEEC15F032C0E4F033C0E5F00001D0
:103B7800E66BE76B6D506E10D8A4C5EF1DF0C7EF6C
:103B88001DF0B0EF1EF080C0D6F081C0D7F082C023
:103B9800D8F083C0D9F0D61FD71FD81FD91FD62B6E
:103BA800000ED723D823D923E451D625DA6FE5515F
:103BB800D721DB6FE651D821DC6FE751D921DD6FC2
:103BC800A00EDA25E06F8C0EDB21E16F000EDC2100
:103BD800E26F000EDD21E36FE3BFFFEF1DF0E3515D
:103BE800E2110BE1A10EE05D8C0EE159D8A0FFEFC8
:103BF8001DF001EF1EF009EF1EF0600EE027730EB6
:103C0800E123FF0EE223FF0EE323E3BF18EF1EF0CC
:103C1800E351E2110BE1510EE05D460EE159D8A0E7
:103C280018EF1EF01AEF1EF020EF1EF0000EDF6FE7
:103C3800000EDE6F26EF1EF0000EDF6F010EDE6F46
:103C480026EF1EF0E7BF37EF1EF0E751E61109E156
:103C5800A00EE45D8C0EE559D8B035EF1EF037EFB5
:103C68001EF0B0EF1EF0DEC018F0DFC019F032EC25
:103C780044F018501910D8B444EF1EF046EF1EF067
:103C8800B0EF1EF0E4C0C6F0E5C0C7F0E6C0C8F06B
:103C9800E7C0C9F098C0CAF099C0CBF08AEC24F00C
:103CA800B0EF1EF0B0EF1EF0B0EF1EF097EC4DF045
:103CB8000009D8B462EF1EF064EF1EF0B0EF1EF0FA
:103CC800000E0001806F000E816F000E826F000EE3
:103CD800836F000E656E000E666E000E676E000E36
:103CE800686EC7EC40F0B0EF1EF0B0EF1EF0B0EF1A
:103CF8001EF07650300AD8B45AEF1EF0010AD8B434
:103D080033EF1DF0020AD8B42AEF1DF0070AD8B421
:103D180045EF1DF0020AD8B43CEF1DF0010AD8B4F3
:103D280057EF1DF00E0AD8B44EEF1DF07A0AD8B43A
:103D38007AEF1DF00D0AD8B460EF1DF0010AD8B46F
:103D48007EEF1DF01F0AD8B469EF1DF0030AD8B43E
:103D580072EF1DF0B0EF1EF012000600FACF04F06B
:103D6800FBCF05F0D9CF06F0DACF07F0F2AABFEF04
:103D78001EF0C1EF1EF08CEF1FF0F2A4C6EF1EF08C
:103D8800C8EF1EF08CEF1FF0F29400018E51010174
:103D9800365D3751800A026E00018F51800A025841
:103DA800D8A0D9EF1EF0DBEF1EF0DEEF1EF0D5969F
:103DB800E1EF1EF0D586E1EF1EF0D8908E35D96E72
:103DC8008F35DA6EC00ED926030EDA22DECF02F066
:103DD800DDCF03F003C002F0036A0250D76ED8901B
:103DE8008E35D96E8F35DA6EC00ED926030EDA22DB
:103DF800DF50D66E98519911D8B405EF1FF007EF30
:103E08001FF010EF1FF080AA0CEF1FF00EEF1FF04D
:103E180022EF1FF010EF1FF098519911D8A417EF57
:103E28001FF019EF1FF030EF1FF084B01EEF1FF0E6
:103E380020EF1FF030EF1FF022EF1FF0000E0101FE
:103E48002C6F000E2D6F000E2E6F000E2F6F010EBF
:103E58000001A96F30EF1FF001012C512D112E1117
:103E68002F11D8B43AEF1FF03CEF1FF082EF1FF08C
:103E78002C07000E2D5B2E5B2F5B02D84DEF1FF039
:103E88000500FA6E3851FD6E3951FE6EFF6AFA5020
:103E98001200010132053311D8A455EF1FF057EF76
:103EA8001FF05DEF1FF0010E1827000E19231A23CB
:103EB8001B232C51185D2D5119592E511A592F5168
:103EC8001B59D8A06AEF1FF06CEF1FF08CEF1FF0A2
:103ED80000018FBF79EF1FF08F5109E1020E8E5D4F
:103EE800D8A079EF1FF07BEF1FF08CEF1FF00101D6
:103EF800326933698CEF1FF08CEF1FF0D59E000EEE
:103F08000001EF6F010EEE6F8CEF1FF08CEF1FF0CA
:103F18009DA091EF1FF093EF1FF02FEF20F09EA0D0
:103F280098EF1FF09AEF1FF02FEF20F0CF0ECF6E13
:103F38002C0ECE6E9E908184010E01012827000E62
:103F480029232A232B230001EE51EF11D8A4AFEF28
:103F58001FF0B1EF1FF011EF20F0010132513311C2
:103F6800D8B4B9EF1FF0BBEF1FF02CEF20F032519F
:103F780000018E270101335100018F238E51010169
:103F8800345D3551800A026E00018F51800A025853
:103F9800D8B0D1EF1FF0D3EF1FF0DEEF1FF034C120
:103FA8008EF035C18FF0000E0101336F000E326FB5
:103FB8002CEF20F000018FBFECEF1FF08F5106E1CE
:103FC8008E05D8B0EAEF1FF0ECEF1FF02CEF20F0D1
:103FD800000E8F6F010E8E6F000E0101336F000E01
:103FE800326F0001A405D8A4FCEF1FF0FEEF1FF00C
:103FF8002CEF20F0000E01012C6F000E2D6F000E2B
:104008002E6F000E2F6F2CEF20F02CEF20F02CEFEE
:1040180020F02CEF20F02CEF20F06F4A702A0101DD
:104028003E4B3F2B320E3E193F11D8A41EEF20F015
:1040380020EF20F02CEF20F0000E516F010E506F92
:10404800000E3F6F000E3E6F2CEF20F02CEF20F09B
:1040580081942FEF20F007C0DAFF06C0D9FF05C012
:10406800FBFF04C0FAFF78921100000E0001A86F50
:10407800000EB56FC851C911D8B445EF20F047EF0D
:1040880020F052EF20F080BA4CEF20F04EEF20F0F5
:1040980052EF20F04C0EB56F52EF20F0C851C91105
:1040A800D8A459EF20F05BEF20F064EF20F084B043
:1040B80060EF20F062EF20F064EF20F04C0EB56F57
:1040C800B551D8A46AEF20F06CEF20F0B6EF21F0DC
:1040D800C7BF73EF20F071EF20F07BEF20F021EEE7
:1040E80067F0DE50C627DD50C72398EF20F00101A6
:1040F80067510001C65DC751800A606E01016851B1
:10410800800A6058D8A08BEF20F08DEF20F098EF50
:1041180020F021EE67F0DE500001C65FDD50C75B7E
:1041280098EF20F098EF20F0C6C06BF0C7C06CF095
:104138006BC01BF06CC01CF067C11DF068C11EF09D
:1041480048EC48F0C6C008F0C7C009F0000E09BE28
:10415800FF0E0A6E0B6E88C00CF089C00DF08AC085
:104168000EF08BC00FF087EC4EF008C014F009C0B9
:1041780015F00AC016F00BC017F021EE67F0DECF7D
:1041880018F0DDCF19F0000E19BEFF0E1A6E1B6E67
:104198002EEC3DF014C0CAF015C0CBF016C0CCF020
:1041A80017C0CDF00001C851C911D8B4DEEF20F016
:1041B800E0EF20F0FFEF20F065C060F066C061F02E
:1041C80067C062F068C063F0601E611E621E631EF5
:1041D800602A000E612262226322CA516024CA6FDB
:1041E800CB516120CB6FCC516220CC6FCD51632075
:1041F800CD6F1CEF21F0CAC060F0CBC061F0CCC01D
:1042080062F0CDC063F0601E611E621E631E602AEC
:10421800000E61226222632265506024CA6F6650D4
:104228006120CB6F67506220CC6F68506320CD6FE0
:10423800CDBF23EF21F021EF21F031EF21F088519C
:10424800CA25CA6F8951CB21CB6F8A51CC21CC6F3B
:104258008B51CD21CD6F63EF21F08851CA5D895113
:10426800CB598A51CC59CD51800A606E8B51800A46
:104278006058D8A042EF21F044EF21F063EF21F01D
:1042880088C060F089C061F08AC062F08BC063F0BA
:10429800601E611E621E631E602A000E6122622279
:1042A8006322CA516024CA6FCB516120CB6FCC51B5
:1042B8006220CC6FCD516320CD6F63EF21F0C851E0
:1042C800C911D8B46AEF21F06CEF21F080EF21F02A
:1042D800CAC055F0CBC056F0CCC057F0CDC058F08E
:1042E800000E5A6E010E596E9EC05BF09FC05CF0C6
:1042F8000EEC2FF094EF21F0CAC055F0CBC056F069
:10430800CCC057F0CDC058F0000E5A6E000E596E52
:104318009EC05BF09FC05CF00EEC2FF094EF21F094
:10432800EDEC4FF0460E0001B519D8B49EEF21F020
:10433800A0EF21F0B6EF21F0B551D8B4A6EF21F0E7
:10434800A8EF21F0B6EF21F0010EA86FC6C046F124
:10435800C7C047F1C8C048F1C9C049F1B6EF21F05C
:10436800B6EF21F052EC37F0809212007650D8A4C4
:10437800C0EF21F0C2EF21F00AEF23F0A2EC50F0D9
:104388000009D8B4CAEF21F0CCEF21F00AEF23F0EE
:104398004E0E766E0AEF23F00AEF23F00AEF23F0B1
:1043A800FF0E6B240001D56FFF0E6C20D66FA8514D
:1043B800D8B4E1EF21F0E3EF21F0F2EF21F00101B1
:1043C80048514911D8A4EBEF21F0EDEF21F0F2EFBD
:1043D80021F00001D54BD62BF2EF21F0D5C0C6F065
:1043E800D6C0C7F0000E0001C96F000EC86F39ECC7
:1043F80020F025EF23F0010E6B240001D56F000E8D
:104408006C20D66FA851D8B40CEF22F00EEF22F032
:104418001EEF22F0010148054911D8A416EF22F039
:1044280018EF22F01EEF22F00001D507D8A0D6071A
:104438001EEF22F0D5C0C6F0D6C0C7F0000E0001AE
:10444800C96F010EC86F39EC20F025EF23F0060E76
:10445800326E040E336E6BC034F06CC035F0FF0E54
:10446800366E020EEEEC15F032C0D5F033C0D6F041
:104478006D506E10D8A443EF22F045EF22F025EFDF
:1044880023F06B500001D51909E16C50D619D8B446
:1044980050EF22F052EF22F025EF23F06BC0CEF060
:1044A8006CC0CFF0CE1FCF1FCE4BCF2B0101675171
:1044B8000001CE27010168510001CF23D551CE2537
:1044C800D36FD651CF21D46FD3510101675D6851A5
:1044D800800A0001CE6FD451800ACE59D8B077EF48
:1044E80022F079EF22F081EF22F021EE67F0DE5022
:1044F800D35FDD50D45B81EF22F00101683568316C
:104508000001CF6F010167310001CE6FD351CE5D3D
:10451800CF51800AD06FD451800AD059D8B097EFC4
:1045280022F099EF22F09FEF22F0000ED26F000EDA
:10453800D16FA5EF22F0000ED26F010ED16FA5EF5B
:1045480022F0010167510001D55DD651800ACE6F76
:1045580001016851800A0001CE59D8B0B6EF22F0A7
:10456800B8EF22F025EF23F0D1C018F0D2C019F02F
:1045780032EC44F018501910D8B4C5EF22F0C7EF48
:1045880022F025EF23F0D5C0C6F0D6C0C7F098C0FA
:10459800C8F099C0C9F039EC20F025EF23F025EFD9
:1045A80023F025EF23F0000E1F6E010E1E6E6DEC3A
:1045B80051F025EF23F024EC46F025EF23F097EC9B
:1045C8004DF00009D8B4EBEF22F0EDEF22F025EF23
:1045D80023F0000E6C6E000E6B6E000E656E000E02
:1045E800666E000E676E000E686E000E0001806F2A
:1045F800000E816F000E826F000E836F1DEC52F06B
:1046080025EF23F025EF23F025EF23F07650300A2D
:10461800D8B4E3EF22F0730AD8B4DFEF22F00D0A22
:10462800D8B4FFEF21F0010AD8B42BEF22F01F0A0B
:10463800D8B4D4EF21F0030AD8B4D7EF22F025EF8D
:1046480023F01200000E0001B56FC851D8B42FEF47
:1046580023F031EF23F03AEF23F080BA36EF23F05E
:1046680038EF23F03AEF23F04C0EB56FC851D8A4B9
:1046780040EF23F042EF23F04BEF23F084B047EFF5
:1046880023F049EF23F04BEF23F04C0EB56FB551F3
:10469800D8A451EF23F053EF23F086EF24F0C7BFDF
:1046A8005AEF23F058EF23F062EF23F021EE69F080
:1046B800DE50C627DD50C7237FEF23F00101695183
:1046C8000001C65DC751800A606E01016A51800A07
:1046D8006058D8A072EF23F074EF23F07FEF23F037
:1046E80021EE69F0DE500001C65FDD50C75B7FEF49
:1046F80023F07FEF23F0C6C040F1C7C041F1010E9F
:10470800010140251B6E000E41211C6E96C01DF054
:1047180097C01EF0000E206E010E1F6E000E226E56
:10472800010E216EF0EC47F0C6C008F0C7C009F0D2
:10473800000E09BEFF0E0A6E0B6E88C00CF089C011
:104748000DF08AC00EF08BC00FF087EC4EF008C059
:1047580014F009C015F00AC016F00BC017F021EECE
:1047680069F0DECF18F0DDCF19F0000E19BEFF0E8C
:104778001A6E1B6E2EEC3DF014C0C9F015C0CAF0BD
:1047880016C0CBF017C0CCF00001C851D8B4CFEF99
:1047980023F0D1EF23F0F0EF23F065C060F066C09E
:1047A80061F067C062F068C063F0601E611E621E3F
:1047B800631E602A000E612262226322C9516024AE
:1047C800C96FCA516120CA6FCB516220CB6FCC51DF
:1047D8006320CC6F0DEF24F0C9C060F0CAC061F04F
:1047E800CBC062F0CCC063F0601E611E621E631E07
:1047F800602A000E61226222632265506024C96F1C
:1048080066506120CA6F67506220CB6F6850632082
:10481800CC6FCCBF14EF24F012EF24F022EF24F079
:104828008851C925C96F8951CA21CA6F8A51CB21BC
:10483800CB6F8B51CC21CC6F56EF24F08851C95DDA
:104848008951CA598A51CB59CC51800A606E8B5113
:10485800800A6058D8A033EF24F035EF24F056EFE3
:1048680024F088C060F089C061F08AC062F08BC013
:1048780063F0601E611E621E631E602A000E6122C4
:1048880062226322C9516024C96FCA516120CA6F6C
:10489800CB516220CB6FCC516320CC6F56EF24F004
:1048A80056EF24F0C851D8B45CEF24F05EEF24F042
:1048B80072EF24F0C9C055F0CAC056F0CBC057F00B
:1048C800CCC058F0000E5A6E010E596E9EC05BF0B7
:1048D8009FC05CF00EEC2FF086EF24F0C9C055F0B5
:1048E800CAC056F0CBC057F0CCC058F0000E5A6E74
:1048F800000E596E9EC05BF09FC05CF00EEC2FF06E
:1049080086EF24F052EC37F080921200000E00017E
:10491800A76F000EB56FCA51CB11D8B496EF24F02B
:1049280098EF24F0A3EF24F080BA9DEF24F09FEFD6
:1049380024F0A3EF24F04C0EB56FA3EF24F0CA5176
:10494800CB11D8A4AAEF24F0ACEF24F0B5EF24F0F3
:1049580084B0B1EF24F0B3EF24F0B5EF24F04C0E9F
:10496800B56FB551D8A4BBEF24F0BDEF24F0E7EF45
:1049780025F0C9BFC4EF24F0C2EF24F0CEEF24F035
:10498800A00EC6278C0EC723000EC823000EC9230D
:10499800EBEF24F0C9BFDDEF24F0C951C8110BE1DA
:1049A800A00EC65D8C0EC759D8A0DDEF24F0DFEF4E
:1049B80024F0EBEF24F0600EC627730EC723FF0E1A
:1049C800C823FF0EC923EBEF24F0EBEF24F0C6C099
:1049D80080F0C7C081F0C8C082F0C9C083F0C6C0EB
:1049E80021F0C7C022F0C8C023F0C9C024F028ECC9
:1049F8004FF021C0CCF022C0CDF023C0CEF024C0AF
:104A0800CFF00001CA51CB11D8B40DEF25F00FEF4C
:104A180025F02EEF25F065C060F066C061F067C034
:104A280062F068C063F0601E611E621E631E602A29
:104A3800000E612262226322CC516024CC6FCD51DA
:104A48006120CD6FCE516220CE6FCF516320CF6FE2
:104A58004BEF25F0CCC060F0CDC061F0CEC062F065
:104A6800CFC063F0601E611E621E631E602A000EC6
:104A780061226222632265506024CC6F66506120F7
:104A8800CD6F67506220CE6F68506320CF6FCFBF65
:104A980052EF25F050EF25F060EF25F08851CC2536
:104AA800CC6F8951CD21CD6F8A51CE21CE6F8B51DC
:104AB800CF21CF6F92EF25F08851CC5D8951CD5928
:104AC8008A51CE59CF51800A606E8B51800A605846
:104AD800D8A071EF25F073EF25F092EF25F088C08C
:104AE80060F089C061F08AC062F08BC063F0601E1C
:104AF800611E621E631E602A000E6122622263220A
:104B0800CC516024CC6FCD516120CD6FCE51622045
:104B1800CE6FCF516320CF6F92EF25F0CA51CB11E2
:104B2800D8B499EF25F09BEF25F0AFEF25F0CCC076
:104B380055F0CDC056F0CEC057F0CFC058F0000E9B
:104B48005A6E010E596E9EC05BF09FC05CF00EEC71
:104B58002FF0C3EF25F0CCC055F0CDC056F0CEC035
:104B680057F0CFC058F0000E5A6E000E596E9EC016
:104B78005BF09FC05CF00EEC2FF0C3EF25F0460E03
:104B88000001B519D8B4CBEF25F0CDEF25F0E7EF4C
:104B980025F0B551D8B4D3EF25F0D5EF25F0E7EFE0
:104BA80025F0010EA76FC6C01CF1C7C01DF1C8C013
:104BB8001EF1C9C01FF1CAC044F1CBC045F1E7EFEF
:104BC80025F0E7EF25F052EC37F0809212001BEF4A
:104BD80027F0000E0101416F000E406F96C042F1B0
:104BE80097C043F1010E0001A56F000E656E000E1F
:104BF800666E000E676E000E686E3BEF27F0000EC3
:104C08000D6E030E93EC51F0B30E106EFD0E116E87
:104C1800F7EC48F0000E0001C66F000EC76F000EDB
:104C2800C86F000EC96FFF0ECB6FCA69B6EC3AF0B9
:104C3800B4EC38F00001B551D8B425EF26F027EFD1
:104C480026F02BEF26F0000EA56F3BEF27F0030EA2
:104C5800A56F3BEF27F03BEF27F0000E0D6E030E1C
:104C680093EC51F0BE0E106EFD0E116EF7EC48F08D
:104C78008CC1C6F08DC1C7F00001C86BC96B4EC1AD
:104C8800CAF04FC1CBF0B6EC3AF00001B551D8B438
:104C980050EF26F052EF26F05FEF26F04C0EB519D4
:104CA800D8B459EF26F05BEF26F05FEF26F0000E40
:104CB800A56F3BEF27F0040EA56F3BEF27F03BEF06
:104CC80027F0000E0D6E030E93EC51F0970E106E48
:104CD800FE0E116EF7EC48F0000E0001C66F000ED4
:104CE800C76F000EC86F000EC96FFF0ECB6FCA6981
:104CF800B6EC3AF00001B551D8B485EF26F087EF4D
:104D080026F094EF26F04C0EB519D8B48EEF26F0A5
:104D180090EF26F094EF26F0000EA56F3BEF27F0FA
:104D2800050EA56F3BEF27F03BEF27F00101420787
:104D3800D8A0430742514311D8A4A5EF26F0A7EF06
:104D480026F0ACEF26F0060E0001A56F3BEF27F02A
:104D5800000E0D6E030E93EC51F03C0E106EFF0E1C
:104D6800116EF7EC48F00101404B412B40C1C6F0F1
:104D780041C1C7F0010E0001C86F26EC23F0000105
:104D8800B551D8B4CAEF26F0CCEF26F0D0EF26F014
:104D9800000EA56F3BEF27F0030EA56F3BEF27F042
:104DA8003BEF27F03BEF27F0000E0D6E030E93EC60
:104DB80051F0350E106EFF0E116EF7EC48F0000141
:104DC80096510101691909E10001975101016A1918
:104DD800D8A4F1EF26F0F3EF26F0FEEF26F0000E50
:104DE8000001C76F000EC66F010EC86F26EC23F0D6
:104DF80009EF27F0000E0001C76F000EC66F000E06
:104E0800C86F26EC23F009EF27F0070E0001A56F05
:104E18003BEF27F0460EB56F52EC37F01AEC4DF029
:104E2800000E0001A56F3BEF27F03BEF27F00001D4
:104E3800A551010AD8B403EF26F0030AD8B4EDEF60
:104E480025F0010AD8B431EF26F0070AD8B465EF87
:104E580026F0010AD8B49AEF26F0030AD8B4D8EF9E
:104E680026F0010AD8B40EEF27F03BEF27F0120026
:104E7800000E756E010E0001B46F000EAE6F000ECD
:104E88009F6F000E9E6F000E0101286F000E296FA4
:104E9800000E2A6F000E2B6F000E0001806F000EAF
:104EA800816F000E826F000E836F000E656E000E1C
:104EB800666E000E676E000E686E000E9D6F000E27
:104EC8009C6F000E9B6F000E9A6F000EB26F010E62
:104ED800B36F000EB56FF2EC52F075C074F0C7EC0A
:104EE80040F00001B151D8B47CEF27F07EEF27F0F5
:104EF8009DEF27F0000E206E020E1F6E75C021F088
:104F0800226A7550030D000EF324236E030EF4205D
:104F1800246E000E256E010E266E0DEC0FF0000EAD
:104F28000D6E020E93EC51F03E0E05EC4BF09DEF2A
:104F380027F00E0E0D6E000E93EC51F0990E106EC8
:104F4800FF0E116EF7EC48F0010E00019E25156E5C
:104F5800000E9F21166E010E176E000E186E57EC8C
:104F68003EF07550030D000EF324D96E030EF420A5
:104F7800DA6EDF500001E26F7CEF28F09EEC19F04A
:104F8800000E0D6E000E93EC51F00001B151D8B433
:104F9800D0EF27F0D2EF27F0DAEF27F0BD0E106E32
:104FA800FF0E116EF7EC48F0E2EF27F0A50E106E39
:104FB800FF0E116EF7EC48F0E2EF27F0000E00014B
:104FC800B56FB151D8B4EBEF27F0EDEF27F008EF4C
:104FD80028F0B151D8B4F3EF27F0F5EF27F000EF40
:104FE80028F04E0E7618D8B4FCEF27F0FEEF27F025
:104FF80008EF28F000EF28F0B251D8B406EF28F0F7
:1050080008EF28F02CEF28F075C074F0D3EC11F0FD
:105018000001B151BFEC4AF00E0E0D6E000E93EC7C
:1050280051F0990E106EFF0E116EF7EC48F0010E5C
:1050380000019E25156E000E9F21166E010E176E3B
:10504800000E186E57EC3EF0C7EC40F02CEF28F03D
:10505800430E7618D8B433EF28F035EF28F041EF37
:1050680028F0430E0001B519D8A43DEF28F03FEF12
:1050780028F046EF28F041EF28F0010EBFEC4AF087
:1050880046EF28F00001B151D8B44DEF28F04FEFAA
:1050980028F05DEF28F04F0E7618D8A456EF28F0C8
:1050A80058EF28F05DEF28F0000EBFEC4AF05DEFF6
:1050B80028F0580E7618D8B464EF28F066EF28F078
:1050C80072EF28F0580E0001B519D8A46EEF28F039
:1050D80070EF28F07CEF28F072EF28F0000E216EB8
:1050E800030E206E9DEC36F087EF28F07CEF28F059
:1050F8000001B351D8A483EF28F085EF28F0C2EF60
:1051080027F087EF28F0000E0001A16F0B0EA06FAB
:105118001200050E5BEC4FF09EEC19F0A5EF29F09C
:10512800030E0001B66F3C0E4CEC49F00001ED6F28
:10513800ED29D8B4A2EF28F0A4EF28F0C5EF29F0A4
:1051480012EC4EF0EDC0C1F09BEC4CF0010E0001EA
:10515800B66FC5EF29F0C5EF29F0070EED19D8B4E1
:10516800B8EF28F0BAEF28F0C0EF28F0000EEB6F88
:10517800020EEA6FC6EF28F0000EEB6F010EEA6F21
:10518800C6EF28F0EAC0ECF0F2EC52F0850E106E93
:10519800F90E116EF7EC48F00001EDA5D6EF28F0F6
:1051A800D8EF28F0E7EF28F0000E0D6EEC5193ECE5
:1051B80051F00001EC2BB60E106EFA0E116EF7ECE2
:1051C80048F0E7EF28F00001EDA3EDEF28F0EFEF4E
:1051D80028F0FEEF28F0000E0D6EEC5193EC51F024
:1051E8000001EC2BA30E106EFA0E116EF7EC48F0CE
:1051F800FEEF28F00001EDA104EF29F006EF29F0F9
:1052080015EF29F0000E0D6EEC5193EC51F00001F2
:10521800EC2BC90E106EFA0E116EF7EC48F015EF74
:1052280029F00001ED51D8A41CEF29F01EEF29F058
:105238002DEF29F0000E0D6EEC5193EC51F00001AA
:10524800EC2BB70E106EFC0E116EF7EC48F02DEF3C
:1052580029F0000E706E000E6F6E020E0001B66F20
:10526800C5EF29F070BE42EF29F02C0E6F5C010EDD
:105278007058D8A042EF29F044EF29F0C5EF29F083
:10528800030EB66FC5EF29F0C5EF29F0F2EC52F026
:10529800B80E106EF70E116EF7EC48F0060E0D6E94
:1052A800010E93EC51F02D0E106EFF0E116EF7ECFF
:1052B80048F0000E0D6E030E93EC51F0710E106E57
:1052C800F90E116EF7EC48F0000E706E000E6F6E5E
:1052D800050E0001B66FC5EF29F070BE7DEF29F00D
:1052E800705009E1960E6F5CD8A07DEF29F07FEF32
:1052F80029F0C5EF29F0060EB66FC5EF29F0C5EF06
:1053080029F0000E04EC38F00001C0BF8EEF29F040
:1053180090EF29F09BEF29F0070EB66F000EA16FF2
:105328000C0EA06FC05121EC53F09BEF29F024EC38
:1053380046F0C5EF29F0F2EC13F0C5EF29F0C5EF00
:1053480029F00001B651000AD8B494EF28F0010AF8
:10535800D8B4B1EF28F0030AD8B436EF29F0010A1F
:10536800D8B44AEF29F0060AD8B471EF29F0030A35
:10537800D8B485EF29F0010AD8B49FEF29F0C5EF1A
:1053880029F01200F2EC52F0090E106EF80E116EB0
:10539800F7EC48F0010E0D6E010E93EC51F0410E42
:1053A800106EFE0E116EF7EC48F00D0E326E040E04
:1053B800336E69C134F06AC135F0FF0E366E010EE6
:1053C800EEEC15F032C069F133C06AF101016ABF31
:1053D800F9EF29F06A5107E1020E695DD8B0F7EFDD
:1053E80029F0F9EF29F0FFEF29F0000E6A6F020E9D
:1053F800696FFFEF29F06D506E10D8B406EF2AF0F0
:1054080008EF2AF00CEF2AF0F5EF2AF0F5EF2AF072
:105418000D0E0D6E010E93EC51F069C115F06AC1C5
:1054280016F0040E176E010E186EAAEC41F0000E6D
:105438000D6E020E93EC51F0CF0E106EFB0E116E36
:10544800F7EC48F069C196F06AC197F0010E0D6E4D
:10545800030E93EC51F0F50E106EFD0E116EF7EC85
:1054680048F00D0E326E040E336E96C034F097C0BD
:1054780035F0FF0E366E030EEEEC15F032C096F0E6
:1054880033C097F0000196510101695D0001975101
:1054980001016A59D8B053EF2AF055EF2AF05BEFB3
:1054A8002AF069C196F06AC197F06DEF2AF0000101
:1054B80096519711D8A463EF2AF065EF2AF06DEFA3
:1054C8002AF0000E976F010E966F6DEF2AF06DEFC0
:1054D8002AF06D506E10D8B474EF2AF076EF2AF0E7
:1054E8007AEF2AF0F5EF2AF0F5EF2AF0F2EC52F015
:1054F800000E0D6E000E93EC51F0FE0E106EFC0EB9
:10550800116EF7EC48F08CC108F08DC109F0000E5F
:105518000B6E640E0A6E91EC4BF008C04DF009C09A
:105528004EF0010E0D6E020E93EC51F04DC015F0C9
:105538004EC016F0020E176E010E186E57EC3EF0B4
:105548008D0E106EFD0E116EF7EC48F04DC008F090
:105558004EC009F0000E0B6E640E0A6E98EC52F005
:10556800081E091E084A092A01018C5108244D6E9B
:105578008D5109204E6E4DC015F04EC016F0020E2A
:10558800176E000E186E57EC3EF0E50E106EFF0E0B
:10559800116EF7EC48F0490E106EFE0E116EF7EC26
:1055A80048F0010E326E040E336E8CC134F08DC19A
:1055B80035F0020E366E020EEEEC15F032C08CF1AC
:1055C80033C08DF16D506E10D8B4EDEF2AF0EFEFC7
:1055D8002AF0F3EF2AF0F5EF2AF0F5EF2AF02AEC9B
:1055E80053F0120023C027F024C028F0D8902736A3
:1055F8002836D8902736283627C02BF028C02CF01C
:105608002D6A2E6A21C027F022C028F0D8902736AC
:105618002836D8902736283627C031F028C032F0EF
:10562800336A346AE90E255C030E2658D8A01FEFAA
:105638002BF021EF2BF027EF2BF0030E266EE80E50
:10564800256E3AEF2BF0265007E1030E255CD8B003
:1056580030EF2BF032EF2BF03AEF2BF0000E266EE6
:10566800030E256E3AEF2BF03AEF2BF0FF0E2524B0
:105678000101346FFF0E2620356F36693769000E39
:10568800336F010E326F000E186F000E196F000E87
:105698001A6F000E1B6F000E00018F6F000E8E6FC9
:1056A800000EA46F000E3A6E000E396EFEEF2BF05E
:1056B80031C027F032C028F033C029F034C02AF0B6
:1056C800271E281E291E2A1E272A000E28222922C4
:1056D8002A222B502724086E2C502820096E2D5082
:1056E80029200A6E2E502A200B6E39C00CF03AC0C1
:1056F8000DF0000E0DBEFF0E0E6E0F6E87EC4EF015
:1057080008C014F009C015F00AC016F00BC017F055
:1057180034C118F035C119F0000E19BEFF0E1A6E0B
:105728001B6EE2EC46F031501424356E32501520D1
:10573800366E33501620376E34501720386E385076
:10574800371009E1800E355C020E3658D8B0AFEF3D
:105758002BF0B1EF2BF0D1EF2BF039C036F13AC076
:1057680037F15C0E146E620E156E020E166E000E88
:10577800176E35C018F036C019F037C01AF038C0A7
:105788001BF0E2EC46F0141E151E144A152A14C02C
:105798002FF015C030F0EDEF2BF0800E146EA00E38
:1057A800156E370E166E020E176E35C018F036C01D
:1057B80019F037C01AF038C01BF0E2EC46F0141E9E
:1057C800151E144A152A14C02FF015C030F0EDEF3D
:1057D8002BF0D8903934D96E3A34DA6EC00ED92607
:1057E800030EDA222FC0DEFF30C0DDFF394A3A2A25
:1057F800FEEF2BF02550395C26503A58D8A007EF19
:105808002CF009EF2CF05CEF2BF00BEF2CF01200D2
:1058180013EF2CF000019C51C65F9D51C75B00013E
:105828009C51C65D9D51C759D8B01DEF2CF01FEF94
:105838002CF00EEF2CF021EF2CF09AC008F09BC052
:1058480009F00A6A0B6A88C00CF089C00DF08AC09A
:105858000EF08BC00FF087EC4EF008C014F009C0B2
:1058680015F00AC016F00BC017F09CC018F09DC0C8
:1058780019F01A6A1B6A2EEC3DF014C0CCF015C062
:10588800CDF016C0CEF017C0CFF0C6C008F0C7C024
:1058980009F00A6A0B6A88C00CF089C00DF08AC04A
:1058A8000EF08BC00FF087EC4EF008C014F009C062
:1058B80015F00AC016F00BC017F09CC018F09DC078
:1058C80019F01A6A1B6A2EEC3DF014C0C8F015C016
:1058D800C9F016C0CAF017C0CBF0CCC060F0CDC07C
:1058E80061F0CEC062F0CFC063F0601E611E621E20
:1058F800631E602A000E6122622263220001C851E1
:105908006024D06FC9516120D16FCA516220D26F13
:10591800CB516320D36FC6C09AF0C7C09BF0B45177
:10592800D8B499EF2CF09BEF2CF0D1EF2CF0D3BF2B
:10593800A0EF2CF0A2EF2CF0B6EF2CF0D0C055F071
:10594800D1C056F0D2C057F0D3C058F0000E5A6EEE
:10595800010E596E9EC05BF09FC05CF00EEC2FF0FC
:1059680010EF2DF00001D0518825556ED1518921B5
:10597800566ED2518A21576ED3518B21586E000E24
:105988005A6E010E596E9EC05BF09FC05CF00EEC23
:105998002FF010EF2DF010EF2DF00001D31FD21FC4
:1059A800D11FD06D000ED123D223D323D3BFDFEF75
:1059B8002CF0E1EF2CF0F5EF2CF0D0C055F0D1C071
:1059C80056F0D2C057F0D3C058F0000E5A6E000EF1
:1059D800596E9EC05BF09FC05CF00EEC2FF010EF8C
:1059E8002DF00001D0518825556ED1518921566E70
:1059F800D2518A21576ED3518B21586E000E5A6EA0
:105A0800000E596E9EC05BF09FC05CF00EEC2FF04C
:105A180010EF2DF010EF2DF0EDEC4FF052EC37F0C9
:105A280080921200000E0001AC6F000E386E000E5E
:105A3800376E38BE29EF2DF0385009E1400E375C3B
:105A4800D8A029EF2DF02BEF2DF02FEF2DF05FEFE1
:105A58002DF05FEF2DF037C008F038C009F0000EC8
:105A68000B6E030E0A6E98EC52F0000E0824D96EE5
:105A7800030E0920DA6EDF50D8A445EF2DF047EF6A
:105A88002DF04BEF2DF05FEF2DF05FEF2DF00001C3
:105A9800AC2B374A382A38BE5BEF2DF0385009E175
:105AA800400E375CD8A05BEF2DF05DEF2DF02FEFA7
:105AB8002DF05FEF2DF074500001AC5DD8B067EFAA
:105AC8002DF069EF2DF06DEF2DF0ACC074F06DEF97
:105AD8002DF0AD51745CD8B074EF2DF076EF2DF049
:105AE8007AEF2DF074C0ADF07AEF2DF074502E6E71
:105AF8002F6AAD51306E316A030E3026000E312206
:105B08002E50305C3150800A326E2F50800A325845
:105B1800D8B091EF2DF093EF2DF098EF2DF0745051
:105B2800FD0FAD6F98EF2DF0AD51030D000EF3246E
:105B3800336E030EF420346E000E386E000E376E8E
:105B480038BEB0EF2DF0385009E1040E375CD8A00C
:105B5800B0EF2DF0B2EF2DF0B6EF2DF016EF2EF0DE
:105B680016EF2EF00001AD513724356E000E3820A7
:105B7800366E37C01FF038C020F035C021F036C06F
:105B880022F033C023F034C024F0AC512E6E2F6ABB
:105B980035502E5C2F50800A306E3650800A3058AF
:105BA800D8A0D9EF2DF0DCEF2DF0010EDDEF2DF0B0
:105BB800000E256E010E266E0DEC0FF0000E0D6E18
:105BC800375093EC51F074502E6E2F6A35502E18C2
:105BD80007E136502F18D8A4F4EF2DF0F6EF2DF08A
:105BE800FBEF2DF03E0E05EC4BF000EF2EF0200EF3
:105BF80005EC4BF000EF2EF0030E3326000E342296
:105C0800374A382A38BE12EF2EF0385009E1040E10
:105C1800375CD8A012EF2EF014EF2EF0B6EF2DF06F
:105C280016EF2EF012000C5008240E6E0D500920AD
:105C38000F6EFF0E0E240101306FFF0E0F20316F23
:105C4800C00E081400018C6FFF0E09148D6FFAEF57
:105C58002EF0000E716E3F0E716435EF2EF037EFA7
:105C68002EF03BEF2EF097EF2EF097EF2EF07150BD
:105C780000018C250E6E000E8D210F6E08500E5CF3
:105C880009500F58D8A04BEF2EF04DEF2EF061EFD2
:105C98002EF071508C250E6E000E8D210F6E0E5059
:105CA8000101305D0F503159D8B05DEF2EF05FEF34
:105CB8002EF07AEF2EF061EF2EF0715000018C2556
:105CC8000E6E000E8D210F6E0EC0F6FF0FC0F7FF8F
:105CD800F86A09007150010D100EF324D96E000EF8
:105CE800F420DA6EF5CFDFFF8CEF2EF00AC0D9FF73
:105CF8000BC0DAFF7150010D100EF324E16E000E97
:105D0800F420E26EDFCFE7FF0A4A0B2A8CEF2EF071
:105D1800712A3F0E716493EF2EF095EF2EF03BEF52
:105D28002EF097EF2EF08CC0F6FF8DC0F7FFF86AC3
:105D3800A68EA69CA684A688550EA76EAA0EA76E48
:105D4800A682A198A694000E0001A26F010EA36F6F
:105D5800EEEF2EF08CC0F6FF8DC0F7FFF86A000E4C
:105D6800716E3F0E7164BBEF2EF0BDEF2EF0C1EFE8
:105D78002EF0D9EF2EF0D9EF2EF00001A251010D2F
:105D8800100EF324D96E000EF420DA6EDF50F56E93
:105D9800A22B0D00712A3F0E7164D5EF2EF0D7EFBC
:105DA8002EF0C1EF2EF0D9EF2EF08CC0F6FF8DC08B
:105DB800F7FFF86A400E00018C27000E8D23A68E8F
:105DC800A69CA684550EA76EAA0EA76EA682A198B9
:105DD800EEEF2EF0A307A329D8A4F5EF2EF0F7EFE6
:105DE8002EF0AEEF2EF0A694FAEF2EF00C50082409
:105DF8000E6E0D5009200F6E0E508C5D0F508D5990
:105E0800D8A009EF2FF00BEF2FF02DEF2EF00DEFAC
:105E18002FF0120094C090F095C091F059505A108C
:105E2800D8A419EF2FF01BEF2FF026EF2FF0010168
:105E38006051552661515622000E5722000E5822F5
:105E480026EF2FF0C7EC40F001017851D8A42FEFCE
:105E58002FF031EF2FF038EF2FF074B102D0829687
:105E680001D082863DEF2FF074B102D0829C01D020
:105E7800828C8082000E0D6E030E93EC51F0360E6C
:105E8800106EFD0E116EF7EC48F0000E0001B56FB4
:105E980075C108F076C109F0000E0B6E0A0E0A6E85
:105EA80098EC52F06F5008245E6E705009205F6EB7
:105EB80060EF2FF060EF2FF05E506F5C7050800A3B
:105EC8005D6E5F50800A5D58D8A06DEF2FF06FEFC0
:105ED8002FF060EF2FF071EF2FF055C03BF056C058
:105EE8003CF057C03DF058C03EF059C03FF05AC092
:105EF80040F05BC041F05CC042F0C3EC32F08BEC88
:105F080042F0020E38183910D8B48DEF2FF08FEF09
:105F18002FF0B5EF2FF059505A10D8A496EF2FF064
:105F280098EF2FF0B5EF2FF060C13BF061C13CF066
:105F38003D6A3E6A59505A10D8B4A5EF2FF0A8EF21
:105F48002FF0010EA9EF2FF0000E3F6E406A5BC0E4
:105F580041F05CC042F0C3EC32F08BEC42F0B5EF9C
:105F68002FF001017851D8A4BCEF2FF0BEEF2FF02D
:105F7800D3EF2FF07451D8B4C4EF2FF0C8EF2FF03F
:105F88005D6A5D2AC9EF2FF05D6A5D465D465D4634
:105F980082505D18F70B5D18826EE7EF2FF0010154
:105FA8007451D8B4DAEF2FF0DEEF2FF05D6A5D2A76
:105FB800DFEF2FF05D6A5D3A5D465D4682505D1801
:105FC800BF0B5D18826E0C0E0001A019A111D8B488
:105FD800F0EF2FF0F2EF2FF0F5EF2FF08092F5EFC2
:105FE8002FF0C7EC40F0000E0D6E030E93EC51F04D
:105FF800490E106EFE0E116EF7EC48F01200000EFE
:106008001F6E010E0001BC6F1E501D100BE1400EEB
:106018001B5C7E0E1C58D8A014EF30F016EF30F041
:1060280068EF30F0810E1B5CEE0E1C58FF0E1D58F9
:10603800FF0E1E58D8A023EF30F025EF30F041EFC7
:1060480030F01BC00DF01CC00EF01DC00FF01EC0BC
:1060580010F0800E116EEE0E126EFF0E136EFF0E14
:10606800146ED9EC3FF00DC01BF00EC01CF00FC031
:106078001DF010C01EF041EF30F0000E0001BC6FA3
:106088001BC00DF01CC00EF01DC00FF01EC010F09C
:10609800400E116E7E0E126E000E136E000E146E00
:1060A800D9EC3FF00DC01BF00EC01CF00FC01DF066
:1060B80010C01EF0F80E106EFF0E116EF7EC48F0CF
:1060C800010E1F6E68EF30F01F50D8A46EEF30F04D
:1060D80070EF30F080EF30F01E501D100BE1700EA5
:1060E8001B5C170E1C58D8A07CEF30F07EEF30F008
:1060F800BCEF30F080EF30F01BC00DF01CC00EF08C
:106108001DC00FF01EC010F0600E116EEA0E126E68
:10611800FF0E136EFF0E146ED9EC3FF00DC01BF08E
:106128000EC01CF00FC01DF010C01EF01BC00DF0FB
:106138001CC00EF01DC00FF01EC010F0700E116EC6
:10614800170E126E000E136E000E146ED9EC3FF08F
:106158000DC01BF00EC01CF00FC01DF010C01EF0CB
:10616800FB0E106EFF0E116EF7EC48F0BCEF30F02E
:106178001BC00DF01CC00EF01DC00FF01EC010F0AB
:10618800E80E116E030E126E000E136E000E146EE2
:10619800D9EC3FF00DC01BF00EC01CF00FC01DF075
:1061A80010C01EF0000E0001BC6F1BC00DF01CC01B
:1061B8000EF01DC00FF01EC010F0640E116E000E20
:1061C800126E000E136E000E146ED9EC3FF00DC067
:1061D8001BF00EC01CF00FC01DF010C01EF0730E97
:1061E80005EC4BF0120020C0BCF08180060E1F6445
:1061F80000EF31F002EF31F01EEF31F01BC00DF06F
:106208001CC00EF01DC00FF01EC010F0400E116E25
:10621800420E126E0F0E136E000E146ED9EC3FF084
:106228000DC01BF00EC01CF00FC01DF010C01EF0FA
:106238001EEF31F0050E1F6424EF31F026EF31F028
:1062480042EF31F01BC00DF01CC00EF01DC00FF066
:106258001EC010F0A00E116E860E126E010E136E87
:10626800000E146ED9EC3FF00DC01BF00EC01CF0F0
:106278000FC01DF010C01EF042EF31F0040E1F6475
:1062880048EF31F04AEF31F066EF31F01BC00DF006
:106298001CC00EF01DC00FF01EC010F0100E116EC5
:1062A800270E126E000E136E000E146ED9EC3FF01E
:1062B8000DC01BF00EC01CF00FC01DF010C01EF06A
:1062C80066EF31F0030E1F646CEF31F06EEF31F0C2
:1062D8008AEF31F01BC00DF01CC00EF01DC00FF08E
:1062E8001EC010F0E80E116E030E126E000E136E33
:1062F800000E146ED9EC3FF00DC01BF00EC01CF060
:106308000FC01DF010C01EF08AEF31F0020E1F649E
:1063180090EF31F092EF31F0AEEF31F01BC00DF09D
:106328001CC00EF01DC00FF01EC010F0640E116EE0
:10633800000E126E000E136E000E146ED9EC3FF0B4
:106348000DC01BF00EC01CF00FC01DF010C01EF0D9
:10635800AEEF31F0010E1F64B4EF31F0B6EF31F05B
:10636800D2EF31F01BC00DF01CC00EF01DC00FF0B5
:106378001EC010F00A0E116E000E126E000E136E83
:10638800000E146ED9EC3FF00DC01BF00EC01CF0CF
:106398000FC01DF010C01EF0D2EF31F0000E00014A
:1063A800BC6F1BC00DF01CC00EF01DC00FF01EC04E
:1063B80010F0010E116E000E126E000E136E000E1C
:1063C800146ED9EC3FF01200010E0001AA6F3FC015
:1063D80098F040C099F03BC02CF13CC02DF13DC075
:1063E8002EF13EC02FF101018651D8A4FEEF31F005
:1063F80001EF32F0010E02EF32F0000E736E7350AF
:106408000008436E4328726E412806E14228D8A44A
:1064180010EF32F012EF32F01EEF32F0000E426E43
:10642800050E416E83C149F084C14AF04B6A4C6A3B
:1064380026EF32F081C149F082C14AF04B6A4C6ABA
:1064480026EF32F07BC13AF17CC13BF17FC14DF0C0
:1064580080C14EF04F6A506A4DC043F04EC044F0C0
:106468004FC045F050C046F0431E441E451E461E10
:10647800432A000E44224522462249504324086EEE
:106488004A504420096E4B5045200A6E4C50462015
:106498000B6E41C00CF042C00DF0000E0DBEFF0E99
:1064A8000E6E0F6E87EC4EF008C014F009C015F0A0
:1064B8000AC016F00BC017F0040E186E000E196E05
:1064C800000E1A6E000E1B6E2EEC3DF04D5014247B
:1064D800516E4E501520526E4F501620536E50502C
:1064E8001720546E21EE7DF0DECF08F0DDCF09F0E5
:1064F800000E09BEFF0E0A6E0B6E51C00CF052C0A2
:106508000DF053C00EF054C00FF087EC4EF008C0E9
:1065180014F009C015F00AC016F00BC017F0100EE1
:10652800186E270E196E000E1A6E000E1B6E2EECDA
:106538003DF014C047F015C048F057C121F058C1CC
:1065480022F051C023F052C024F047C008F048C0E0
:1065580009F0000E0B6E0A0E0A6E98EC52F008C095
:1065680025F009C026F0F6EC2AF0000E0001A96F0C
:10657800000EEF6F000EEE6FFDEC44F01200000EFF
:106588000001AA6F3FC098F040C099F094C008F08D
:1065980095C009F00A6A0B6A3BC00CF03CC00DF0CC
:1065A8003DC00EF03EC00FF087EC4EF008C02CF155
:1065B80009C02DF10AC02EF10BC02FF10101735152
:1065C800D8A4E9EF32F0ECEF32F0010EEDEF32F043
:1065D800000E736E73500008436E4328726E57C1E5
:1065E8003AF158C13BF15DC147F05EC148F0496AD4
:1065F8004A6A5BC14DF05CC14EF04F6A506A4DC0AB
:1066080043F04EC044F04FC045F050C046F0431E22
:10661800441E451E461E432A000E44224522462299
:1066280047504324086E48504420096E495045207D
:106638000A6E4A5046200B6E41C00CF042C00DF065
:10664800000E0DBEFF0E0E6E0F6E87EC4EF008C0EA
:1066580014F009C015F00AC016F00BC017F0040EAC
:10666800186E000E196E000E1A6E000E1B6E2EECC0
:106678003DF04D501424516E4E501520526E4F501F
:106688001620536E50501720546E21EE59F0DECF6D
:1066980008F0DDCF09F0000E09BEFF0E0A6E0B6E82
:1066A80051C00CF052C00DF053C00EF054C00FF0A2
:1066B80087EC4EF008C014F009C015F00AC016F0B7
:1066C8000BC017F0100E186E270E196E000E1A6EFA
:1066D800000E1B6E2EEC3DF014C04BF015C04CF0B4
:1066E80057C121F058C122F051C023F052C024F004
:1066F8004BC008F04CC009F0000E0B6E0A0E0A6E73
:1067080098EC52F008C025F009C026F0F6EC2AF003
:10671800000E0001A96F000EEF6F000EEE6F61EC26
:1067280045F0120001017A51D8A49DEF33F09FEF94
:1067380033F0ABEF33F04C0EF66EEF0EF76E000E43
:10674800F86E0800F550556E566AB7EF33F04B0EE9
:10675800F66EEF0EF76E000EF86E0800F550556EE7
:10676800566AB7EF33F055C059F07A51D8A4BFEF45
:1067780033F0C1EF33F0C7EF33F0E80E576E010E78
:10678800586E4BEF34F0000E576E020E586E4BEFFA
:1067980034F04BEF34F031EC0CF0100E0001A0197E
:1067A800A111D8A4DAEF33F0DCEF33F05EEF34F068
:1067B80009EC00F05EEF34F05EEF34F00001924B2C
:1067C800932B93BFEAEF33F0ECEF33F000EF34F0A4
:1067D8005950526E536A5250925D9351800A546ECA
:1067E8005350800A5458D8A0FCEF33F0FEEF33F032
:1067F80006EF34F000EF34F0000E936F000E926F46
:1068080006EF34F092515724D96E93515820DA6E1E
:10681800DF50A66F09EC00F05EEF34F0000192073C
:10682800D8A0930793BF1BEF34F01DEF34F031EF7E
:1068380034F05950526E536A5250925D9351800A07
:10684800546E5350800A5458D8A02DEF34F02FEFCF
:1068580034F039EF34F031EF34F0FF0E5924926FF1
:10686800936BFF0E932339EF34F092515724D96E6E
:1068780093515820DA6EDF50A66F09EC00F05EEFF6
:1068880034F024EC46F05EEF34F05EEF34F07650EE
:10689800430AD8B445EF34F00D0AD8B4E2EF33F028
:1068A800010AD8B4CFEF33F01F0AD8B412EF34F08E
:1068B8005EEF34F0120022C008F023C009F024C0B3
:1068C8000AF025C00BF0680E0C6E010E0D6E000E5E
:1068D8000E6E000E0F6E87EC4EF008C02AF009C04D
:1068E8002BF00AC02CF00BC02DF02AC014F02BC0DE
:1068F80015F02CC016F02DC017F088C018F089C00C
:1069080019F08AC01AF08BC01BF02EEC3DF014C0B1
:106918002EF015C02FF016C030F017C031F02EC081
:1069280008F02FC009F030C00AF031C00BF088C061
:106938000CF089C00DF08AC00EF08BC00FF087EC08
:106948004EF0081E091E0A1E0B1E082A000E0922F8
:106958000A220B222A500824326E2B500920336E4B
:106968002C500A20346E2D500B20356E32C008F0A2
:1069780033C009F034C00AF035C00BF0640E0C6E59
:10698800000E0D6E000E0E6E000E0F6E87EC4EF0B0
:1069980008C014F009C015F00AC016F00BC017F0B3
:1069A80088C018F089C019F08AC01AF08BC01BF093
:1069B8002EEC3DF014C032F015C033F016C034F0A0
:1069C80017C035F035BEF4EF34F0355034103310BD
:1069D80009E1640E325CD8A0F4EF34F0F6EF34F03D
:1069E80006EF35F0000E326E000E336E000E346E78
:1069F800000E356E010E2E26000E2F223022312277
:106A080006EF35F026C00DF0285093EC51F02EC05B
:106A180015F02FC016F0030E176E010E186E57EC06
:106A28003EF02E0E05EC4BF032C015F033C016F0D8
:106A3800020E176E000E186E57EC3EF01200516EE3
:106A48004D0E4F6EEF0E506E000E6E6E000E6D6E98
:106A5800F2EC52F0090E516434EF35F036EF35F0B0
:106A68005BEF35F0B10E106EFF0E116EF7EC48F0CB
:106A7800000E0D6E010E93EC51F00C0E106EFD0E13
:106A8800116EF7EC48F0010EC8EC3DF00E0E326EB8
:106A9800010E336EB0C034F0356A630E366E010EE7
:106AA800EEEC15F032500001B06F65EF35F01F0EB7
:106AB800106EFC0E116EF7EC48F051C0B0F065EFA7
:106AC80035F0000E0D6E030E93EC51F06D506E1004
:106AD800D8A471EF35F073EF35F0BEEF35F0000153
:106AE800B051C00DF3504F26F4505022000E536E93
:106AF800000E526E53BE8AEF35F0535009E1C00EB6
:106B0800525CD8A08AEF35F08CEF35F090EF35F075
:106B1800B6EF35F0B6EF35F052504F244D6E535066
:106B280050204E6E4DC0F6FF4EC0F7FFF86A000EBB
:106B38005224D96E030E5320DA6E0800F5CFDFFF1A
:106B4800524A532A53BEB2EF35F0535009E1C00EF2
:106B5800525CD8A0B2EF35F0B4EF35F090EF35F0D5
:106B6800B6EF35F0900E106EFA0E116EF7EC48F095
:106B7800C6EF35F0490E106EF90E116EF7EC48F0BD
:106B8800C6EF35F0000E706E000E6F6ECEEF35F06A
:106B9800CEEF35F070BEDAEF35F0705009E1960EA1
:106BA8006F5CD8A0DAEF35F0DCEF35F0CEEF35F0DA
:106BB800DEEF35F0000E0001A16F0B0EA06F120082
:106BC80085EF36F084B0EBEF35F0EDEF35F0F2EF0E
:106BD80035F04C0E0001B56F14EF36F0F2EC52F0C0
:106BE8008F0E106EFD0E116EF7EC48F0000E1C6E45
:106BF800030E1B6E18EC4CF0000E556EF00E566E20
:106C0800FF0E576EFF0E586E000E5A6E000E596E2C
:106C18009EC05BF09FC05CF00EEC2FF014EF36F0D6
:106C280052EC37F0000E0001A16F090EA06F9CEF27
:106C380036F080BA22EF36F024EF36F029EF36F03E
:106C48004C0E0001B56F4BEF36F0F2EC52F08F0EA0
:106C5800106EFD0E116EF7EC48F0000E1C6E030E60
:106C68001B6E18EC4CF0000E556EF00E566EFF0EB3
:106C7800576EFF0E586E000E5A6E010E596E9EC06A
:106C88005BF09FC05CF00EEC2FF04BEF36F052EC4F
:106C980037F0000E0001A16F090EA06F9CEF36F0CF
:106CA800000E1F6E030E1E6E6DEC51F09CEF36F059
:106CB80024EC46F09CEF36F097EC4DF00009D8B480
:106CC80068EF36F06AEF36F09CEF36F0000E000100
:106CD800A16F090EA06F000E656E000E666E000EA5
:106CE800676E000E686E000E806F000E816F000EDA
:106CF800826F000E836F9CEF36F09CEF36F09CEFAE
:106D080036F07650300AD8B460EF36F0730AD8B44B
:106D18005CEF36F00D0AD8B41DEF36F01E0AD8B471
:106D2800E6EF35F0030AD8B454EF36F09CEF36F0AE
:106D38001200F2EC52F0000E0D6E000E93EC51F0C2
:106D4800FCEF36F0FD0E106EFE0E116EF7EC48F0FB
:106D58008A0E106EFC0E116EF7EC48F022EF37F039
:106D6800FD0E106EFE0E116EF7EC48F00F0E106E51
:106D7800FC0E116EF7EC48F022EF37F0FD0E106EA6
:106D8800FE0E116EF7EC48F0F90E106EF60E116E4D
:106D9800F7EC48F022EF37F0000E106EFE0E116E81
:106DA800F7EC48F08E0E106EFB0E116EF7EC48F003
:106DB80022EF37F0FD0E106EFE0E116EF7EC48F064
:106DC800500E106EFD0E116EF7EC48F022EF37F002
:106DD800000E106EFE0E116EF7EC48F05A0E106E93
:106DE800FB0E116EF7EC48F022EF37F022EF37F088
:106DF80020C022F021C023F02350000AD8B407EFA6
:106E080037F022EF37F02250000AD8B4A6EF36F058
:106E1800010AD8B4B4EF36F0030AD8B4C2EF36F09A
:106E2800010AD8B4D0EF36F0070AD8B4DEEF36F04E
:106E3800010AD8B4ECEF36F022EF37F09F0E106E4F
:106E4800FF0E116EF7EC48F028C11BF029C11CF0A9
:106E58002AC11DF02BC11EF003EC30F0000E00011A
:106E6800B36F000E0D6E030E93EC51F0F90E106E19
:106E7800F80E116EF7EC48F046EF37F09EEC19F07B
:106E880046EF37F04F0E7618D8A44DEF37F04FEF96
:106E980037F042EF37F051EF37F01200010E2B6E4A
:106EA8002C0E2A6E000E0D6E030E93EC51F0C0EFFF
:106EB80037F0440E106EFA0E116EF7EC48F0EDEC58
:106EC8004FF0000E2B6E640E2A6ED4EF37F0F80EDA
:106ED800106EF90E116EF7EC48F0EDEC4FF0000E65
:106EE8002B6E640E2A6ED4EF37F080BA7EEF37F03F
:106EF80080EF37F08FEF37F084B085EF37F087EF0A
:106F080037F08FEF37F00B0E106EFA0E116EF7ECAC
:106F180048F0D4EF37F080BA94EF37F096EF37F0B7
:106F28009EEF37F01E0E106EFA0E116EF7EC48F059
:106F3800D4EF37F0310E106EFA0E116EF7EC48F000
:106F4800D4EF37F0D4EF37F0D4EF37F0E50E106E0A
:106F5800F90E116EF7EC48F0D4EF37F0490E106EC9
:106F6800FE0E116EF7EC48F0000E2B6E000E2A6E26
:106F7800D4EF37F0D4EF37F00001B551430AD8B455
:106F88006BEF37F0050AD8B4AAEF37F00A0AD8B47D
:106F980079EF37F0140AD8B45DEF37F0B2EF37F075
:106FA800000E706E000E6F6E9EEC19F0E0EF37F079
:106FB8009EEC19F0E0EF37F02A506F5C2B507058B8
:106FC800D8B0E9EF37F0EBEF37F0F8EF37F0430ED2
:106FD8007618D8A4F2EF37F0F4EF37F0DCEF37F09B
:106FE800F8EF37F0F8EF37F0000E0D6E030E93EC64
:106FF80051F0490E106EFE0E116EF7EC48F01200BB
:107008004F6E12EC4EF04F50D8A40DEF38F00FEF42
:1070180038F01CEF38F00001BFBF15EF38F017EF5C
:1070280038F01CEF38F0BFC069F06A6A81EF38F0B9
:10703800F2EC52F05D0E106EFC0E116EF7EC48F09B
:10704800010E0D6E020E93EC51F0850E106EFE0EC1
:10705800116EF7EC48F0010E0001C225506E516A1E
:10706800000E512238EF38F00B0E326E010E336EDF
:1070780050C034F051C035F0FF0E366E020EEEEC03
:1070880015F032C069F033C06AF06ABE57EF38F0C5
:107098006A5007E1060E695CD8B055EF38F057EF33
:1070A80038F038EF38F06ABE62EF38F06A5008E11D
:1070B8006904D8A062EF38F064EF38F038EF38F0A0
:1070C80066EF38F06906D8A06A060001C2514D6E15
:1070D8004E6A69504D1809E16A504E18D8B477EFD6
:1070E80038F079EF38F081EF38F069C0C2F09BECE6
:1070F8004CF081EF38F081EF38F069C00EF06AC0CB
:107108000FF0DBEC4CF0F00E0101551909E1DE0E31
:107118005619D8B492EF38F094EF38F09AEF38F067
:107128001BEC42F02AEC53F09AEF38F06FC108F0EC
:1071380070C109F071C10AF072C10BF04EEC4EF04B
:107148008AC124F18BC125F10101266B276B000E42
:10715800656E000E666E000E676E000E686E120099
:1071680060C158F061C159F001017851D8A4BFEF4E
:1071780038F0C1EF38F0C8EF38F074B102D0829619
:1071880001D08286CFEF38F074B102D0829C01D052
:10719800828CCFEF38F0000E0001B56F75C108F092
:1071A80076C109F0000E0B6E0A0E0A6E98EC52F0CA
:1071B8006F500824566E70500920576EE6EF38F06D
:1071C800E6EF38F056506F5C7050800A556E575095
:1071D800800A5558D8A0F3EF38F0F5EF38F0E6EF0D
:1071E80038F0F7EF38F058C03BF059C03CF0000ECB
:1071F8003CBEFF0E3D6E3E6E000E406E000E3F6EB2
:10720800000E426E000E416EC3EC32F08BEC42F081
:10721800020E38183910D8B414EF39F016EF39F0D7
:107228002AEF39F060C13BF061C13CF03D6A3E6A2B
:10723800000E406E010E3F6E000E426E000E416E53
:10724800C3EC32F08BEC42F02AEF39F001017851AF
:10725800D8A431EF39F033EF39F048EF39F07451F1
:10726800D8B439EF39F03DEF39F0556A552A3EEF79
:1072780039F0556A55465546554682505518F70B0C
:107288005518826E5EEF39F001017451D8B44FEF92
:1072980039F053EF39F0556A552A54EF39F0556AE9
:1072A800553A5546554682505518BF0B5518826EAB
:1072B8005EEF39F0C7EC40F012002D6EFF0E22246D
:1072C800306E316AFF0E312231BE6FEF39F06DEF4B
:1072D80039F073EF39F0CCEF39F0CCEF39F023C047
:1072E80014F024C015F025C016F026C017F00A0EB9
:1072F800186E000E196E000E1A6E000E1B6EE2EC70
:1073080046F014C02EF015C02FF02EC008F02FC084
:1073180009F0000E0B6E0A0E0A6E98EC52F0081E69
:10732800091E084A092A235008242E6E24500920D1
:107338002F6E23C014F024C015F025C016F026C007
:1073480017F00A0E186E000E196E000E1A6E000E57
:107358001B6EE2EC46F014C023F015C024F016C0F2
:1073680025F017C026F030502824D96E3150292036
:10737800DA6E2E50300FDF6E3006D8A0310631BEDF
:10738800CAEF39F0C8EF39F073EF39F0CCEF39F0C4
:1073980021C00DF02D5093EC51F0000E316E000E0F
:1073A800306EF8EF39F027502A6E2B6A30502A18C1
:1073B80007E131502B18D8A4E4EF39F0E6EF39F0A3
:1073C800EBEF39F02E0E05EC4BF0EBEF39F03050C7
:1073D8002824D96E31502920DA6EDF5005EC4BF0A5
:1073E800304A312AF8EF39F022502A6E2B6A2A5097
:1073F800305C3150800A2C6E2B50800A2C58D8A053
:1074080008EF3AF00AEF3AF0D7EF39F00CEF3AF01C
:107418001200000E096EFA0E086E000E0B6E320E88
:107428000A6EE8EC49F03F0E0001AC611EEF3AF03D
:1074380020EF3AF0B3EF3AF0000E406E3F0E3F6E89
:1074480093EF3AF03FC008F040C009F0000E0B6E11
:10745800030E0A6E98EC52F008C041F009C042F0E1
:10746800FD0E396EFF0E3A6E41C03BF042C03CF053
:1074780039503B263A503C22000E3B24D96E030E6D
:107488003C20DA6E000E4124E16E030E4220E26ECB
:10749800DFCFE7FFFE0E396EFF0E3A6E41C03BF0BC
:1074A80042C03CF039503B263A503C22000E3B2467
:1074B800D96E030E3C20DA6E010E41243D6E000E9B
:1074C80042203E6E000E3D24E16E030E3E20E26E29
:1074D800DFCFE7FFFF0E396EFF0E3A6E41C03BF07B
:1074E80042C03CF039503B263A503C22000E3B2427
:1074F800D96E030E3C20DA6E020E41243D6E000E5A
:1075080042203E6E000E3D24E16E030E3E20E26EE8
:10751800DFCFE7FF3F06D8A0400693EF3AF074505C
:10752800396E3A6A3F50395C3A50800A3B6E405097
:10753800800A3B58D8A0A3EF3AF0A5EF3AF026EF1F
:107548003AF0A7EF3AF07450030D000EF324D96E09
:10755800030EF420DA6E190EDF6EB3EF3AF016EC74
:107568002DF01200C6C021F0C7C022F0C8C023F019
:10757800C9C024F0F5EC4EF021C0CEF022C0CFF007
:1075880023C0D0F024C0D1F0000E0001B56FCE5159
:10759800845DCF518559D05186598751800A606ED4
:1075A800D151800A6058D8B0DCEF3AF0DEEF3AF0FB
:1075B8000CEF3BF0000ECD6F010ECC6F84C060F075
:1075C80085C061F086C062F087C063F0601E611EEE
:1075D800621E631E602A000E612262226322CE515F
:1075E8006024CE6FCF516120CF6FD0516220D06F11
:1075F800D1516320D16F80BA04EF3BF006EF3BF026
:1076080038EF3BF04C0EB56F38EF3BF038EF3BF0FE
:10761800000ECD6F000ECC6FCEC060F0CFC061F011
:10762800D0C062F0D1C063F0601E611E621E631E8E
:10763800602A000E61226222632284516024CE6F88
:1076480085516120CF6F86516220D06F87516320AA
:10765800D16F84B032EF3BF034EF3BF038EF3BF0C2
:107668004C0EB56F38EF3BF0B551D8A43EEF3BF068
:1076780040EF3BF052EF3BF0CEC055F0CFC056F094
:10768800D0C057F0D1C058F0CCC059F0CDC05AF096
:10769800CAC05BF0CBC05CF056EC3BF052EC37F064
:1076A8008092120001017851D8A45DEF3BF05FEFA2
:1076B8003BF066EF3BF087B102D0829C01D0828C10
:1076C8006BEF3BF087B102D0829601D08286808230
:1076D800000E0001B56F88C108F089C109F0000EDD
:1076E8000B6E0A0E0A6E98EC52F06F5008245E6E0C
:1076F800705009205F6E83EF3BF083EF3BF05E50E4
:107708006F5C7050800A5D6E5F50800A5D58D8A02B
:1077180090EF3BF092EF3BF083EF3BF094EF3BF0C0
:1077280055C03BF056C03CF057C03DF058C03EF045
:1077380059C03FF05AC040F05BC041F05CC042F015
:10774800E8EC31F08BEC42F001017851D8A4AFEFAE
:107758003BF0B1EF3BF0C6EF3BF08751D8B4B7EF41
:107768003BF0BBEF3BF05D6A5D2ABCEF3BF05D6A26
:107778005D3A5D465D4682505D18BF0B5D18826EAE
:10778800DAEF3BF001018751D8B4CDEF3BF0D1EFF0
:107798003BF05D6A5D2AD2EF3BF05D6A5D465D466F
:1077A8005D4682505D18F70B5D18826E0C0E000165
:1077B800A019A111D8B4E3EF3BF0E5EF3BF0E8EFF7
:1077C8003BF08092E8EF3BF0000E0D6E030E93EC59
:1077D80051F0490E106EFE0E116EF7EC48F01200D3
:1077E80026C00DF0285093EC51F07C0E106EFE0E62
:1077F800116EF7EC48F022C008F023C009F024C04D
:107808000AF025C00BF0100E0C6E270E0D6E000E40
:107818000E6E000E0F6E87EC4EF008C02AF009C0FD
:107828002BF00AC02CF00BC02DF02AC014F02BC08E
:1078380015F02CC016F02DC017F024C118F025C182
:1078480019F026C11AF027C11BF02EEC3DF014C028
:1078580032F015C033F016C034F017C035F032C01E
:1078680014F033C015F034C016F035C017F0640EAC
:10787800186E000E196E000E1A6E000E1B6E2EEC9E
:107888003DF014C02EF015C02FF016C030F017C010
:1078980031F02EC008F02FC009F030C00AF031C016
:1078A8000BF0640E0C6E000E0D6E000E0E6E000EC8
:1078B8000F6E87EC4EF0081E091E0A1E0B1E082AC2
:1078C800000E09220A220B2232500824326E33504D
:1078D8000920336E34500A20346E35500B20356E33
:1078E8002EC015F02FC016F0030E176E010E186E7D
:1078F80057EC3EF02E0E05EC4BF032C015F033C0BD
:1079080016F0020E176E000E186E57EC3EF0E60EDB
:10791800106EFF0E116EF7EC48F01200000E096EA3
:10792800FA0E086E000E0B6E320E0A6EE8EC49F085
:107938007450030D000EF324D96E030EF420DA6E92
:10794800DF50D8B4AAEF3CF0ACEF3CF02BEF3DF0A1
:1079580074C03DF03E6A3EBEBBEF3CF03E5009E1CC
:107968003E0E3D5CD8A0BBEF3CF0BDEF3CF0C1EF54
:107978003CF02BEF3DF02BEF3DF03DC008F03EC052
:1079880009F0000E0B6E030E0A6E98EC52F008C058
:107998003FF009C040F0030E3F24396E000E40202E
:1079A8003A6E000E3924D96E030E3A20DA6E000EB4
:1079B8003F24E16E030E4020E26EDFCFE7FF040EA6
:1079C8003F24396E000E40203A6E000E3924D96EDD
:1079D800030E3A20DA6E010E3F243B6E000E402063
:1079E8003C6E000E3B24E16E030E3C20E26EDFCFBE
:1079F800E7FF050E3F24396E000E40203A6E000E58
:107A08003924D96E030E3A20DA6E020E3F243B6EFB
:107A1800000E40203C6E000E3B24E16E030E3C201D
:107A2800E26EDFCFE7FF3D4A3E2A3EBE25EF3DF03E
:107A38003E5009E13E0E3D5CD8A025EF3DF027EF12
:107A48003DF0C1EF3CF02BEF3DF02BEF3DF016EC95
:107A58002DF01200000E1D6E1BBE37EF3DF035EF06
:107A68003DF043EF3DF01B1E1A1E191E186C000E48
:107A780019221A221B22010E1D6E43EF3DF017BE7C
:107A88004AEF3DF048EF3DF056EF3DF0171E161E49
:107A9800151E146C000E152216221722010E1D1A2F
:107AA80056EF3DF0000E1E6E000E1F6E000E206E8B
:107AB800000E216E185019101A101B10D8B467EF59
:107AC8003DF069EF3DF0ABEF3DF0010E1C6E75EF38
:107AD8003DF0D890183619361A361B361C2A75EF21
:107AE8003DF01BAE7AEF3DF07CEF3DF06DEF3DF0E1
:107AF80080EF3DF080EF3DF0D8901E361F362036DF
:107B080021361850145C195015581A5016581B5025
:107B18001758D8A092EF3DF094EF3DF09FEF3DF05D
:107B28001850145E1950155A1A50165A1B50175AE5
:107B38001E809FEF3DF0D8901B321A32193218324E
:107B48001C2E80EF3DF0ABEF3DF0ABEF3DF01D504C
:107B5800D8B4B1EF3DF0B3EF3DF0BDEF3DF0211EDD
:107B6800201E1F1E1E6C000E1F2220222122BDEF88
:107B78003DF01EC014F01FC015F020C016F021C043
:107B880017F0C7EF3DF01200196E4D0E176EEF0E8D
:107B9800186E000E0D6E030E93EC51F01950D8B408
:107BA800D8EF3DF0DAEF3DF0E2EF3DF0150E106E44
:107BB800FF0E116EF7EC48F0EAEF3DF01D0E106E67
:107BC800FF0E116EF7EC48F0EAEF3DF0000E1B6E69
:107BD800090E1B64F2EF3DF0F4EF3DF0F8EF3DF0D5
:107BE80053EF3EF053EF3EF0000E166E000E156E8A
:107BF800000E1A6E3F0E1A6404EF3EF006EF3EF0D8
:107C08000AEF3EF023EF3EF023EF3EF017C0F6FFF9
:107C180018C0F7FFF86A0800F5501526000E16225E
:107C2800030E1726000E18221A2A3F0E1A641FEF99
:107C38003EF021EF3EF00AEF3EF023EF3EF0155004
:107C48001610D8A42AEF3EF02DEF3EF0010E2EEFCD
:107C58003EF0000E136E146A1950131A000E141A0F
:107C680013501410D8B43BEF3EF03DEF3EF042EF16
:107C78003EF0200E05EC4BF048EF3EF01B50300F65
:107C880005EC4BF048EF3EF01B2A090E1B644FEF42
:107C98003EF051EF3EF0F8EF3DF053EF3EF05D0E51
:107CA80005EC4BF0120018C0BCF0818016BE61EFE5
:107CB8003EF05FEF3EF06AEF3EF02D0E05EC4BF024
:107CC800156C161ED8B0162A6AEF3EF015C019F0CA
:107CD80016C01AF0040E176474EF3EF076EF3EF00B
:107CE80086EF3EF019C00DF01AC00EF0270E106E88
:107CF800100E0F6EC3EC45F00DC019F00EC01AF04F
:107D080086EF3EF0030E17648CEF3EF08EEF3EF0E8
:107D18009EEF3EF019C00DF01AC00EF0030E106E63
:107D2800E80E0F6EC3EC45F00DC019F00EC01AF046
:107D38009EEF3EF0020E1764A4EF3EF0A6EF3EF071
:107D4800B6EF3EF019C00DF01AC00EF0000E106E1E
:107D5800640E0F6EC3EC45F00DC019F00EC01AF09A
:107D6800B6EF3EF0010E1764BCEF3EF0BEEF3EF0FA
:107D7800CEEF3EF019C00DF01AC00EF0000E106ED6
:107D88000A0E0F6EC3EC45F00DC019F00EC01AF0C4
:107D9800CEEF3EF0000E0001BC6F19C00DF01AC006
:107DA8000EF0000E106E010E0F6EC3EC45F01200BF
:107DB80044EF3FF00001AA51D8B4E5EF3EF0E7EFF9
:107DC8003EF05AEF3FF084C022F085C023F086C011
:107DD80024F087C025F0000E276E010E266E000ED7
:107DE800296E020E286EF4EC3BF05AEF3FF05AEF82
:107DF8003FF00001AA51D8B404EF3FF006EF3FF07E
:107E08001AEF3FF084C022F085C023F086C024F02A
:107E180087C025F0000E276E010E266E000E296E13
:107E2800020E286EF4EC3BF02EEF3FF065C022F016
:107E380066C023F067C024F068C025F0000E276EE6
:107E4800070E266E000E296E010E286E5FEC34F0C8
:107E58002EEF3FF065C022F066C023F067C024F023
:107E680068C025F0000E276E070E266E000E296EDC
:107E7800010E286E5FEC34F05AEF3FF05AEF3FF0F6
:107E8800A0C036F0A1C037F03750000AD8B44FEF81
:107E98003FF02EEF3FF03650060AD8B4DEEF3EF042
:107EA8000A0AD8B4FDEF3EF02EEF3FF01200000EA4
:107EB800506E030E516E4D0E526EEF0E536EF2EC75
:107EC80052F0B70E106EFF0E116EF7EC48F0000E70
:107ED8000D6E010E93EC51F00C0E106EFD0E116E2E
:107EE800F7EC48F0000EC8EC3DF00E0E326E010EB5
:107EF800336EB0C034F0356A630E366E010EEEECA8
:107F080015F032500001B06F000E0D6E030E93ECA9
:107F180051F06D506E10D8A494EF3FF096EF3FF0FB
:107F2800B3EF3FF00001B051C00DF3505226F450AA
:107F3800532252C008F053C009F050C00AF051C093
:107F48000BF0000E0D6EC00E0C6E17EC2EF0900E9E
:107F5800106EFA0E116EF7EC48F0BBEF3FF0490EC9
:107F6800106EF90E116EF7EC48F0BBEF3FF0000E03
:107F7800706E000E6F6EC3EF3FF0C3EF3FF070BE40
:107F8800CFEF3FF0705009E1960E6F5CD8A0CFEFAD
:107F98003FF0D1EF3FF0C3EF3FF0D3EF3FF0000EDB
:107FA8000001A16F0B0EA06F1200000E1A6E000EDA
:107FB800196E090E1964E3EF3FF0E5EF3FF0E9EFC2
:107FC8003FF025EF40F025EF40F011500D5C1250C6
:107FD8000E5813500F5814501058D8A0F6EF3FF011
:107FE800F8EF3FF025EF40F01A2A11C015F012C043
:107FF80016F013C017F014C018F0151E161E171E21
:10800800181E152A000E1622172218220D501524A4
:108018000D6E0E5016200E6E0F5017200F6E10505A
:108028001820106E1AEF40F025EF40F0192A090EBB
:10803800196421EF40F023EF40F0E9EF3FF025EF1E
:1080480040F01A50D8A42BEF40F02DEF40F038EF55
:1080580040F00001BC51D8A434EF40F036EF40F0B6
:1080680041EF40F038EF40F01A50300F05EC4BF07C
:10807800000E0001BC6F46EF40F0200E05EC4BF0FF
:1080880046EF40F00DC00DF00EC00EF00FC00FF01F
:1080980010C010F050EF40F01200000E0D6E0BBE35
:1080A8005AEF40F058EF40F062EF40F00A6C0B1EB8
:1080B800D8B00B2A010E0D6E62EF40F009BE69EFD1
:1080C80040F067EF40F071EF40F0086C091ED8B03F
:1080D800092A010E0D1A71EF40F0000E0F6E000E06
:1080E8000E6E0A500B10D8B47CEF40F07EEF40F0D3
:1080F800B2EF40F0010E0C6E88EF40F0D8900A36CF
:108108000B360C2A88EF40F00BAE8DEF40F08FEF66
:1081180040F082EF40F093EF40F093EF40F0D890BA
:108128000E360F360A50085C0B500958D8A09FEF3E
:1081380040F0A1EF40F0A8EF40F00A50085E0B5065
:10814800095A0E80A8EF40F0D8900B320A320C2E54
:1081580093EF40F0B2EF40F0B2EF40F00D50D8B4DA
:10816800B8EF40F0BAEF40F0C0EF40F00E6C0F1ED1
:10817800D8B00F2AC0EF40F00EC008F00FC009F0C9
:10818800C6EF40F01200060E0001A019A111D8B4E4
:10819800D0EF40F0D2EF40F038EF41F0010E0D6E15
:1081A800010E93EC51F0660E106EFF0E116EF7EC97
:1081B80048F080C014F081C015F082C016F083C06A
:1081C80017F0640E186E000E196E000E1A6E000E6F
:1081D8001B6E2EEC3DF014C026F015C027F016C01B
:1081E80028F017C029F026C008F027C009F028C0D9
:1081F8000AF029C00BF0640E0C6E000E0D6E000E16
:108208000E6E000E0F6E87EC4EF0081E091E0A1E39
:108218000B1E082A000E09220A220B220001805197
:108228000824226E81510920236E82510A20246E6F
:1082380083510B20256E26C015F027C016F0030EBB
:10824800176E010E186E57EC3EF02E0E05EC4BF033
:1082580022C015F023C016F0020E176E000E186E1D
:1082680057EC3EF038EF41F012008190320E5BEC93
:108278004FF0300E816E8182080E0D6E4BEF41F08B
:1082880000F000F000F000F000F000F000F00D2E1B
:1082980044EF41F08192140E5BEC4FF08182080E9E
:1082A8000E6E5EEF41F000F000F000F000F000F01C
:1082B80000F000F00E2E57EF41F08192140E5BECA7
:1082C8004FF08182080E0F6E71EF41F000F000F060
:1082D80000F000F000F000F000F00F2E6AEF41F01F
:1082E8008192140E5BEC4FF0200E816E8182080E95
:1082F800106E86EF41F000F000F000F000F000F0A2
:1083080000F000F0102E7FEF41F08192640E116EA4
:1083180095EF41F000F000F000F000F000F000F000
:1083280000F0112E8EEF41F09AEF41F0280ED5ECB7
:108338004BF0080ED5EC4BF00C0ED5EC4BF0060EBE
:10834800D5EC4BF0FA0E5BEC4FF0120018C0BCF005
:108358008180040E1764B3EF41F0B5EF41F0C5EF2B
:1083680041F015C00DF016C00EF0270E106E100E5D
:108378000F6EC3EC45F00DC015F00EC016F0C5EF3A
:1083880041F0030E1764CBEF41F0CDEF41F0DDEF84
:1083980041F015C00DF016C00EF0030E106EE80E79
:1083A8000F6EC3EC45F00DC015F00EC016F0DDEFF2
:1083B80041F0020E1764E3EF41F0E5EF41F0F5EF0D
:1083C80041F015C00DF016C00EF0000E106E640ED0
:1083D8000F6EC3EC45F00DC015F00EC016F0F5EFAA
:1083E80041F0010E1764FBEF41F0FDEF41F00DEF96
:1083F80042F015C00DF016C00EF0000E106E0A0EF9
:108408000F6EC3EC45F00DC015F00EC016F00DEF61
:1084180042F0000E0001BC6F15C00DF016C00EF042
:10842800000E106E010E0F6EC3EC45F01200DE0E4A
:108438000101566FF00E556F000E586F960E576F6C
:10844800000E5A6F140E596F010E5C6FF40E5B6FBD
:10845800070E5E6FD00E5D6F000E5F6F000E616FCE
:108468000A0E606F000E626F040E636F040E646F75
:10847800010E656F000E686F3C0E676FB80E6B6F6C
:108488000B0E6C6F000E6D6F000E6E6FA00E6F6F8F
:108498008C0E706F000E716F000E726F010E736F8D
:1084A800000E746F000E766F000E756F000E896FE8
:1084B800000E886F000E776F000E786F800E796F50
:1084C800000E7A6F000E7C6F640E7B6F000E7E6F5D
:1084D800140E7D6F000E806F640E7F6F030E826F27
:1084E800E80E816F070E846FD00E836F010E866FC2
:1084F800000E856F1F0E8B6F400E8A6F0F0E8D6FEB
:10850800A00E8C6F000E6A6F1E0E696F1200000EAF
:108518003B6E000E3A6ED6EF42F0DCEC3EF09EEC7D
:1085280019F0C9EF42F0D59E000E0001EF6F010E61
:10853800EE6F000E01012C6F000E2D6F000E2E6FD6
:10854800000E2F6F580E0001B56F000E3B6E020E25
:108558003A6ED6EF42F00C0E0001A019A111D8B462
:10856800B8EF42F0BAEF42F0C2EF42F031EC53F00C
:10857800000E3B6E010E3A6EC2EF42F0430E000150
:10858800B56FD6EF42F0D6EF42F07650430AD8B432
:10859800AFEF42F01B0AD8B497EF42F0D6EF42F0A3
:1085A800D6EF42F00001EE51EF11D8B4DEEF42F001
:1085B800E0EF42F091EF42F0E2EF42F0A951D8B477
:1085C800E8EF42F0EAEF42F0F2EF42F04C0EB56FFE
:1085D800000E3B6E020E3A6EF2EF42F03AC038F0EF
:1085E8003BC039F0F8EF42F012004EEF43F00001C3
:1085F800AC51745CD8B003EF43F005EF43F008EFDB
:1086080043F0742A08EF43F016EC2DF061EF43F0C5
:108618007450D8B412EF43F014EF43F017EF43F05F
:10862800740617EF43F016EC2DF061EF43F0960E49
:10863800176E430E8DEC4FF00009D8B426EF43F0C7
:1086480028EF43F02CEF43F092EC3CF061EF43F05D
:10865800000E0001A16F0B0EA06F61EF43F061EFF8
:1086680043F0960E176E4F0E8DEC4FF00009D8B4FC
:1086780040EF43F042EF43F046EF43F00DEC3AF0A1
:1086880061EF43F059EC4DF061EF43F061EF43F0D7
:1086980061EF43F07650430AD8B41BEF43F00D0A5C
:1086A800D8B4FBEF42F0010AD8B435EF43F01F0A03
:1086B800D8B40CEF43F061EF43F012000101785198
:1086C800D8A469EF43F06BEF43F072EF43F073B057
:1086D80002D0829E01D0828E79EF43F073B002D02F
:1086E800829A01D0828A79EF43F000019007D8A0DE
:1086F800910791BF8AEF43F0915106E19005D8B0F8
:1087080088EF43F08AEF43F0B3EF43F094C090F062
:1087180095C091F0010E6526000E66226722682238
:108728008851655C895166588A5167586850800A33
:10873800016E8B51800A0158D8A0A5EF43F0A7EF2E
:1087480043F0B3EF43F08851655E8951665A8A5108
:10875800675A8B51685AB3EF43F0B3EF43F0010106
:108768007851D8A4BAEF43F0BCEF43F0C3EF43F01D
:1087780072B002D0829E01D0828ECAEF43F072B0EE
:1087880002D0829A01D0828ACAEF43F01200000E0A
:108798000F6E000E0E6E0FBEDBEF43F00F5009E1B7
:1087A800400E0E5CD8A0DBEF43F0DDEF43F0E1EFC5
:1087B80043F031EF44F031EF44F00EC008F00FC041
:1087C80009F0000E0B6E030E0A6E98EC52F0000EC4
:1087D8000824D96E030E0920DA6E000EDF6E0EC073
:1087E80008F00FC009F0000E0B6E030E0A6E98EC2D
:1087F80052F0010E0826000E0922000E0824D96E38
:10880800030E0920DA6E000EDF6E0EC008F00FC0EE
:1088180009F0000E0B6E030E0A6E98EC52F0020E71
:108828000826000E0922000E0824D96E030E09201E
:10883800DA6E000EDF6E0E4A0F2A0FBE2DEF44F0DF
:108848000F5009E1400E0E5CD8A02DEF44F02FEF39
:1088580044F0E1EF43F031EF44F01200000E0D6EEA
:10886800030E93EC51F0590E106EF80E116EF7ECE2
:1088780048F03FEF44F09EEC19F073EF44F0000E1F
:108888000001996F010E986F000E196E010E186E97
:1088980097EF44F097EF44F0000E0001996F000E37
:1088A800986F000E196E010E186E97EF44F097EF4F
:1088B80044F018C098F019C099F0000E196E010E16
:1088C800186E97EF44F097EF44F0000E196E000E03
:1088D800186E97EF44F097EF44F03FEF44F076506E
:1088E800430AD8B469EF44F00D0AD8B443EF44F012
:1088F800010AD8B45DEF44F01F0AD8B450EF44F031
:108908003FEF44F03FEF44F03FEF44F0000E106EAD
:10891800140E116E030E1EEC51F0000E196E000EAF
:10892800186E97EF44F012000EC008F00FC009F05F
:10893800000E0B6E390E0A6E98EC52F0060E0824E3
:10894800146E000E0920156E000E136E390E126E8D
:10895800550E166E010E176E000E196E000E186E6B
:10896800EFEF44F016C0D9FF17C0DAFF18501424EF
:10897800086E19501520096E0BEC53F0116EDE507D
:108988001118D8B4CAEF44F0CCEF44F0E9EF44F042
:1089980018501424086E19501520096E16C0D9FFF6
:1089A80017C0DAFFDF500A6E3BEC52F0185014245F
:1089B800086E19501520096E0BEC53F016C0D9FF3C
:1089C80017C0DAFFDF6EE9EF44F0184A192A164A91
:1089D800172AEFEF44F01250185C13501958D8A01A
:1089E800F8EF44F0FAEF44F0B6EF44F0FCEF44F04F
:1089F8001200010E0001AA6F98519911D8B407EF1F
:108A080045F009EF45F03EEF45F0960E0101386F4D
:108A1800960E396F7851D8A414EF45F016EF45F04B
:108A280029EF45F08551D8B41CEF45F020EF45F00B
:108A3800086A082A21EF45F0086A083A825008189F
:108A4800EF0B0818826E59EF45F001018551D8B433
:108A580030EF45F034EF45F0086A082A35EF45F065
:108A6800086A82500818FE0B0818826E59EF45F004
:108A780059EF45F0600E0101386F940E396F785147
:108A8800D8A449EF45F04BEF45F052EF45F085B1DA
:108A980002D0829801D0828859EF45F085B102D082
:108AA800829001D0828059EF45F0D586F00ED76EBE
:108AB800F00ED66EF28AD58E1200000198519911E7
:108AC800D8B469EF45F06BEF45F0A0EF45F0C40E60
:108AD8000101386F860E396F7851D8A476EF45F0CA
:108AE80078EF45F08AEF45F05F51D8B47EEF45F056
:108AF80082EF45F0086A082A83EF45F0086A825039
:108B08000818FE0B0818826EBBEF45F001015F5193
:108B1800D8B491EF45F095EF45F0086A082A96EF2A
:108B280045F0086A083A82500818EF0B0818826E58
:108B3800BBEF45F0BBEF45F0060E0101386F8D0E17
:108B4800396F7851D8A4ABEF45F0ADEF45F0B4EFED
:108B580045F05FB102D0829001D08280BBEF45F032
:108B68005FB102D0829801D08288BBEF45F0D586EC
:108B7800F00ED76EF00ED66EF28AD58E1200000E69
:108B8800146E000E136E090E1364CDEF45F0CFEF8F
:108B980045F0D3EF45F0FCEF45F0FCEF45F00F5002
:108BA8000D5C10500E58D8A0DCEF45F0DEEF45F014
:108BB800FCEF45F0142A0FC011F010C012F0111E7E
:108BC800121E114A122A0D5011240D6E0E50122039
:108BD8000E6EF1EF45F0FCEF45F0132A090E136411
:108BE800F8EF45F0FAEF45F0D3EF45F0FCEF45F02C
:108BF8001450D8A402EF46F004EF46F00FEF46F009
:108C08000001BC51D8A40BEF46F00DEF46F018EF69
:108C180046F00FEF46F01450300F05EC4BF0000E05
:108C28000001BC6F1DEF46F0200E05EC4BF01DEF68
:108C380046F00DC00DF00EC00EF023EF46F0120006
:108C4800F2EC52F06D0E106EF80E116EF7EC48F063
:108C58006950310F05EC4BF0000E0D6E010E93ECD0
:108C680051F07D0E106EFA0E116EF7EC48F0450EBD
:108C7800106EF80E116EF7EC48F0010179AF47EF6E
:108C880046F049EF46F062EF46F07AAF4EEF46F015
:108C980050EF46F058EF46F0810E106EF80E116E48
:108CA800F7EC48F07BEF46F0A90E106EF80E116E47
:108CB800F7EC48F07BEF46F07BEF46F07AAF67EFD2
:108CC80046F069EF46F071EF46F0950E106EF80E1B
:108CD800116EF7EC48F07BEF46F09F0E106EF80E21
:108CE800116EF7EC48F07BEF46F07BEF46F0070E8D
:108CF8000001B66F000EA16F000EA06F12000101F7
:108D08007851D8A48AEF46F08CEF46F093EF46F0FE
:108D180073B002D0829E01D0828E9AEF46F073B073
:108D280002D0829A01D0828A9AEF46F00001900719
:108D3800D8A0910791BFABEF46F0915106E190059D
:108D4800D8B0A9EF46F0ABEF46F0CAEF46F094C0B2
:108D580090F095C091F0FF0E6526FF0E6622FF0E7B
:108D68006722FF0E682268BEBEEF46F0BCEF46F0F1
:108D7800CAEF46F088516526895166228A516722D2
:108D88008B516822CAEF46F0CAEF46F001017851CC
:108D9800D8A4D1EF46F0D3EF46F0DAEF46F072B040
:108DA80002D0829E01D0828EE1EF46F072B002D0EE
:108DB800829A01D0828AE1EF46F01200000E1C6E02
:108DC800000E1D6E000E1E6E000E1F6E185019103C
:108DD8001A101B10D8B4F3EF46F0F5EF46F035EF54
:108DE80047F0010E206E01EF47F0D890183619367B
:108DF8001A361B36202A01EF47F01BAE06EF47F064
:108E080008EF47F0F9EF46F00CEF47F00CEF47F0AA
:108E1800D8901C361D361E361F361850145C195053
:108E280015581A5016581B501758D8A01EEF47F05F
:108E380020EF47F02BEF47F01850145E1950155AE1
:108E48001A50165A1B50175A1C802BEF47F0D8900F
:108E58001B321A3219321832202E0CEF47F035EF38
:108E680047F01CC014F01DC015F01EC016F01FC03E
:108E780017F012000001A551D8B445EF47F047EFAD
:108E880047F082EF47F0EBEC25F097EF47F082EFE1
:108E980047F0020E0001A56F97EF47F0C1EC52F0C2
:108EA80097EF47F024EC46F097EF47F097EC4DF03A
:108EB8000009D8B462EF47F064EF47F097EF47F046
:108EC800000E0101416F000E406F000E656E000E2E
:108ED800666E000E676E000E686E000E0001806FF1
:108EE800000E816F000E826F000E836F1AEC4DF03A
:108EF80097EF47F097EF47F097EF47F07650300A33
:108F0800D8B45AEF47F0730AD8B456EF47F00C0AB2
:108F1800D8B44DEF47F01C0AD8B452EF47F097EF9A
:108F280047F097EF47F01200F2EC52F01D0E106E6A
:108F3800F80E116EF7EC48F0000E0D6E020E93EC71
:108F480051F0DF0E106EFB0E116EF7EC48F00A0EB2
:108F5800326E050E336E6BC134F06CC135F0030E02
:108F6800366E020EEEEC15F032C06BF133C06CF1C8
:108F780001016D6B6E6BC9EF47F0600E6B27730EC6
:108F88006C23FF0E6D23FF0E6E236EBFDAEF47F0E2
:108F98006E516D1109E1A10E6B5D8C0E6C59D8B044
:108FA800D8EF47F0DAEF47F0C1EF47F0DCEF47F0D2
:108FB800000E0001806F000E816F000E826F000EA0
:108FC800836F000E656E000E666E000E676E000EF3
:108FD800686E2AEC53F01200010E236EE80E1D5C39
:108FE800030E1E58D8A0FBEF47F0FDEF47F000EF47
:108FF80048F0232A00EF48F01E5009E1640E1D5C7A
:10900800D8A009EF48F00BEF48F00EEF48F0232AFC
:109018000EEF48F01E5009E10A0E1D5CD8A017EFAC
:1090280048F019EF48F01CEF48F0232A1CEF48F0ED
:1090380021C00DF01F5093EC51F0F50E106EFE0E8E
:10904800116EF7EC48F01BC015F01CC016F023C0D9
:1090580017F0010E186E57EC3EF0D20E106EFF0E90
:10906800116EF7EC48F01DC015F01EC016F023C0B5
:1090780017F0010E186E57EC3EF0490E106EFE0EFA
:10908800116EF7EC48F01200010E1F6EE80E1D5C21
:10909800030E1E58D8A053EF48F055EF48F058EF8C
:1090A80048F01F2A58EF48F01E5009E1640E1D5C75
:1090B800D8A061EF48F063EF48F066EF48F01F2A48
:1090C80066EF48F01E5009E10A0E1D5CD8A06FEF4C
:1090D80048F071EF48F074EF48F01F2A74EF48F039
:1090E800010E0D6E020E93EC51F0930E106EFF0EF2
:1090F800116EF7EC48F01BC015F01CC016F0040EFA
:10910800176E010E186E57EC3EF0D20E106EFF0E61
:10911800116EF7EC48F01DC015F01EC016F01FC008
:1091280017F0010E186E57EC3EF0490E106EFE0E49
:10913800116EF7EC48F012006BC114F06CC115F019
:109148006DC116F06EC117F0640E186E000E196E20
:10915800000E1A6E000E1B6E2EEC3DF014C022F0AD
:1091680015C023F0010E0D6E020E93EC51F05F0E48
:10917800106EFF0E116EF7EC48F022C015F023C0F8
:1091880016F0030E176E010E186E57EC3EF08D0E9A
:10919800106EFD0E116EF7EC48F022C008F023C0E7
:1091A80009F0000E0B6E640E0A6E98EC52F0081E61
:1091B800091E084A092A01016B510824226E6C51C4
:1091C8000920236E22C015F023C016F0020E176E78
:1091D800000E186E57EC3EF0490E106EFE0E116E22
:1091E800F7EC48F0120081803AEF49F010C0F6FF22
:1091F80011C0F7FFF86A0800F5500A0AD8A407EF6B
:1092080049F009EF49F029EF49F012EF49F012EF60
:1092180049F0200ED5EC4BF012EF49F00001B82BC5
:10922800B805126E130E12641CEF49F01EEF49F0D8
:109238000DEF49F020EF49F0000E0D6EB72993ECC1
:1092480051F0104A112A3AEF49F010C0F6FF11C048
:10925800F7FFF86A0800F550D5EC4BF0104A112AD0
:109268000001B82B3AEF49F03AEF49F010C0F6FF89
:1092780011C0F7FFF86A0800F5500009D8A447EFB5
:1092880049F049EF49F0FAEF48F04BEF49F0120086
:109298001D6EC1C01EF01F68000E0001C16F9EEC5C
:1092A80019F0206E2050D8B45CEF49F05EEF49F019
:1092B80099EF49F01DC017F020508DEC4FF00009D0
:1092C800D8B469EF49F06BEF49F099EF49F0000E17
:1092D800216E070E216473EF49F075EF49F079EFBD
:1092E80049F099EF49F099EF49F02150010D9E0E90
:1092F800F324D96E010EF420DA6E2050DE18D8A4BB
:1093080088EF49F08AEF49F08EEF49F021C01FF04D
:1093180099EF49F0212A070E216495EF49F097EF5C
:1093280049F079EF49F099EF49F01EC0C1F01F509C
:109338009EEF49F01200C8EF49F0000E0001B16F2E
:109348003CEC27F0E7EF49F0010E0001B16F3CEC6F
:1093580027F0E7EF49F0D2EC52F0E7EF49F0CBEC19
:1093680043F0D2EC52F0E7EF49F0FF0E23EC35F072
:10937800E7EF49F05BEC3FF0E7EF49F024EC46F00B
:10938800E7EF49F0E7EF49F07650310AD8B4A1EF9A
:1093980049F0030AD8B4A8EF49F0010AD8B4AFEFEE
:1093A80049F0070AD8B4B3EF49F0010AD8B4B9EFC5
:1093B80049F0030AD8B4BEEF49F0750AD8B4C2EF31
:1093C80049F0E7EF49F012000001EE51EF11D8B46F
:1093D800F0EF49F0F2EF49F02FEF4AF0000E106E6F
:1093E800000E0F6E1CEF4AF0818608C00DF004EFE6
:1093F8004AF000F000F000F000F000F000F000F09B
:109408000D2EFDEF49F0819608C00EF013EF4AF0DB
:1094180000F000F000F000F000F000F000F00E2E78
:109428000CEF4AF018EF4AF00F4A102A1CEF4AF0E6
:109438000A500F5C1050800A0C6E0B50800A0C58B2
:10944800D8A029EF4AF02BEF4AF0F8EF49F02FEFB8
:109458004AF02FEF4AF0120001017851D8A437EFF3
:109468004AF039EF4AF040EF4AF073B002D0829ADE
:1094780001D0828A47EF4AF073B002D0829E01D0B1
:10948800828E47EF4AF0FF0E00018427FF0E8523E6
:10949800FF0E8623FF0E8723020E016E5BEF4AF054
:1094A80000F000F000F000F000F000F000F0012EF5
:1094B80054EF4AF060EF4AF001017851D8A467EF01
:1094C8004AF069EF4AF070EF4AF072B002D0829A1F
:1094D80001D0828A77EF4AF072B002D0829E01D022
:1094E800828E77EF4AF01200EE0EF66EA00EF76E3F
:1094F800000EF86E02EE00F010EE55F00900F5CF00
:10950800EEFFE550E150FAE1800EF66E9D0EF76E23
:10951800000EF86E01EE8EF010EE69F00900F5CF3E
:10952800EEFFE550E150FAE103EEC0F017EED0F09F
:10953800EE6AE550E150FCE1E250FAE103EE00F09A
:10954800C00EEE6AE806FDE101EE00F08E0EEE6A4E
:10955800E806FDE100EE80F0460EEE6AE806FDE161
:1095680000EE65F0130EEE6AE806FDE17890789259
:109578000001BEEF4FF02F6E010E2E6E2FC0B1F01E
:109588000001B151D8B4CBEF4AF0CDEF4AF0ECEF7F
:109598004AF0000E206E030E1F6E75C021F0226A7D
:1095A8007550030D000EF324236E030EF420246E71
:1095B800000E256E010E266E0DEC0FF0000E0D6EDE
:1095C800030E93EC51F03E0E05EC4BF004EF4BF01C
:1095D80000019C519D11D8B4F4EF4AF0F6EF4AF01F
:1095E80004EF4BF09AC01BF09BC01CF09CC01DF010
:1095F8009DC01EF048EC48F004EF4BF004EF4BF030
:1096080012000C6E81800CC008F0F00E0816815014
:109618000F0B0810816E8182080E096E1BEF4BF04C
:1096280000F000F000F000F000F000F000F0092E6B
:1096380014EF4BF081920CC008F0083AF00E0816AF
:1096480081500F0B0810816E8182080E0A6E34EF6C
:109658004BF000F000F000F000F000F000F000F037
:109668000A2E2DEF4BF08192640E0B6E43EF4BF0F8
:1096780000F000F000F000F000F000F000F00B2E19
:109688003CEF4BF048EF4BF00001B82B1200010102
:109698007851D8A452EF4BF054EF4BF05BEF4BF0FE
:1096A80073B002D0829A01D0828A62EF4BF073B015
:1096B80002D0829E01D0828E62EF4BF0010E000133
:1096C8008427000E852386238723020E016E74EFFC
:1096D8004BF000F000F000F000F000F000F000F0B7
:1096E800012E6DEF4BF079EF4BF001017851D8A4C2
:1096F80080EF4BF082EF4BF089EF4BF072B002D065
:10970800829A01D0828A90EF4BF072B002D0829E8A
:1097180001D0828E90EF4BF01200000E0E6E000EFC
:109728000D6E0A500B10D8B49CEF4BF09EEF4BF027
:10973800D0EF4BF0010E0C6EA8EF4BF0D8900A3624
:109748000B360C2AA8EF4BF00BAEADEF4BF0AFEF9A
:109758004BF0A2EF4BF0B3EF4BF0B3EF4BF0D890D8
:109768000D360E360A50085C0B500958D8A0BFEFCA
:109778004BF0C1EF4BF0C8EF4BF00A50085E0B50AE
:10978800095A0D80C8EF4BF0D8900B320A320C2ED4
:10979800B3EF4BF0D0EF4BF00DC008F00EC009F05E
:1097A80012000C6E0CC008F0F00E081681500F0B5A
:1097B8000810816E8182080E096EEAEF4BF000F006
:1097C80000F000F000F000F000F000F0092EE3EFE8
:1097D8004BF081920CC008F0083AF00E0816815040
:1097E8000F0B0810816E8182080E0A6E03EF4CF091
:1097F80000F000F000F000F000F000F000F00A2E99
:10980800FCEF4BF08192640E0B6E12EF4CF000F0FF
:1098180000F000F000F000F000F000F00B2E0BEF6D
:109828004CF017EF4CF01200620E1B24D96E010E9B
:109838001C20DA6E040EDF6424EF4CF026EF4CF0A7
:109848002EEF4CF0620E1B24D96E010E1C20DA6E2E
:10985800040EDF6E620E1B24D96E010E1C20DA6E18
:10986800DF501D6E1D5000019E6F9F6B0E0E0D6E1A
:10987800000E93EC51F0990E106EFF0E116EF7EC7E
:1098880048F0620E1B24D96E010E1C20DA6EDF50E0
:109898001D6E010E1D24156E166A000E1622010E8D
:1098A800176E000E186E57EC3EF012009268000E0C
:1098B800806E000E936E000E816E000E946E000E88
:1098C800826E0F0EC16EF00E956E000E836E949030
:1098D800949E9496928092929284928A96800C0E8C
:1098E800BD6E7F0EBE6ECB68040ECA6E9492C6889B
:1098F800C79CC79EC69ACF0ECF6E2C0ECE6ECD805B
:10990800CD92310ECD6E9D80F28CCD88CD8AD59CBE
:10991800D586D580D582D584D59AD768D668D59E80
:10992800F28EF28E39EC41F0F2EC52F01200BE0EDB
:109938000001BE6FEF0EBD6F060E0D6EBD0E0E6EF2
:10994800000E0F6E000E106ECFEF4CF00EC0D9FF58
:109958000FC0DAFF10C008F0096A0BEC53F00C6E68
:10996800DE500C18D8B4BBEF4CF0BDEF4CF0CAEF8A
:109978004CF010C008F0096A0EC0D9FF0FC0DAFF1A
:10998800DF500A6E3BEC52F0CAEF4CF0102A0E4A38
:109998000F2ACFEF4CF00D50105CD8A0D6EF4CF04A
:1099A800D8EF4CF0AAEF4CF0DAEF4CF012000EC0F2
:1099B80008F00FC009F0000E0B6E390E0A6E98EC15
:1099C80052F0060E0824126E000E0920136E000EC7
:1099D800116E390E106E550E146E010E156E000EB6
:1099E800176E000E166E0CEF4DF012501624086E0E
:1099F80013501720096E0BEC53F014C0D9FF15C093
:109A0800DAFFDF6E164A172A144A152A0CEF4DF0B2
:109A18001050165C11501758D8A015EF4DF017EFDD
:109A28004DF0F9EF4CF019EF4DF01200F2EC52F056
:109A38007B0E106EFF0E116EF7EC48F0010E6B24D2
:109A48001B6E000E6C201C6E96C01DF097C01EF099
:109A5800000E206E010E1F6E000E226E010E216E8A
:109A6800F0EC47F084C022F085C023F086C024F0D3
:109A780087C025F0000E276E010E266E000E296E97
:109A8800020E286EF4EC3BF0000E0001A56FCCEC42
:109A980050F0000E0D6E030E93EC51F0CD0E106ECB
:109AA800F70E116EF7EC48F012007450030D000E1B
:109AB800F3242E6E030EF4202F6EF2EC52F02EC01B
:109AC800D9FF2FC0DAFFDF500001C36F20EE01F08D
:109AD8002E50D9262F50DA22DF50C46F20EE02F024
:109AE8002E50D9262F50DA22DF50C56FFF0E106E88
:109AF800FB0E116EF7EC48F0000E206E020E1F6E82
:109B080074C021F0226AC30E236E000E246E000E6C
:109B1800256E010E266E0DEC0FF0000E0001A16FF0
:109B28000E0EA06F12001868000E0D6E030E93EC57
:109B380051F0A30E106EF70E116EF7EC48F0C0EF5F
:109B48004DF09EEC19F0B3EF4DF0010E186EC0EF1A
:109B58004DF0000E186EC0EF4DF0C0EF4DF076508E
:109B6800430AD8B4ADEF4DF00C0AD8B4A9EF4DF0C4
:109B7800C0EF4DF0C0EF4DF01828D8B4C6EF4DF047
:109B8800C8EF4DF0A5EF4DF0CAEF4DF0000E106E86
:109B9800140E116E030E1EEC51F01850D4EF4DF058
:109BA80012001BC008F01CC009F0000E0B6E640EFA
:109BB8000A6E91EC4BF008C01DF009C01EF01DC0E4
:109BC80015F01EC016F0030E176E010E186E57EC36
:109BD8003EF08D0E106EFD0E116EF7EC48F01DC0B4
:109BE80008F01EC009F0000E0B6E640E0A6E98ECA9
:109BF80052F0081E091E084A092A1B5008241D6E27
:109C08001C5009201E6E1DC015F01EC016F0020E55
:109C1800176E000E186E57EC3EF01200060E0D6E11
:109C2800BD0E0B6E000E0C6E000E0E6E2BEF4EF07E
:109C38000EC008F0096A0BEC53F00BC0D9FF0CC03A
:109C4800DAFFDF6E0E2A0B4A0C2A2BEF4EF00D506E
:109C58000E5CD8A032EF4EF034EF4EF01CEF4EF011
:109C680036EF4EF0EF0E0001BD1909E1BE0EBE1928
:109C7800D8B441EF4EF043EF4EF04DEF4EF0800E6A
:109C8800BF6F800EC06F000EC16F000EC26F4DEF28
:109C98004EF012000C680D680E680F6808C088F056
:109CA80009C089F00AC08AF00BC08BF0000E0001D1
:109CB800956F010E946F6EEF4EF08B358B338A33B0
:109CC80089338833D89094379537D8900C360D3629
:109CD8000E360F368BBF7BEF4EF08B5106E18A05AF
:109CE800D8B079EF4EF07BEF4EF061EF4EF07DEF9C
:109CF8004EF00C5001016F170D5070170E50711770
:109D08000F5072171200000E106E000E116E000E2A
:109D1800126E000E136E91EF4EF008A096EF4EF003
:109D280098EF4EF0A2EF4EF00C5010260D50112275
:109D38000E5012220F501322A2EF4EF0D8900C367C
:109D48000D360E360F36D8900B320A3209320832E9
:109D5800085009100A100B10D8A4B5EF4EF0B7EF51
:109D68004EF091EF4EF010C008F011C009F012C08B
:109D78000AF013C00BF01200D801C801B801A801FD
:109D880045023502250215023233304E3458374F1A
:109D9800010053333231583635344F393837434E52
:109DA800305031323353343536583738394F5030D4
:109DB8004E43434E30504F39383758363534533385
:109DC800323150304E433738394F343536583132C6
:109DD8003353000102030405060B0C140708090A93
:019DE8001565
:109DEA0024C108F025C109F026C10AF027C10BF0E9
:109DFA0021C00CF022C00DF023C00EF024C00FF0D9
:109E0A0087EC4EF0880E0824146E130E0920156E86
:109E1A00000E0A20166E000E0B20176E100E186E1A
:109E2A00270E196E000E1A6E000E1B6EE2EC46F03B
:109E3A0014C021F015C022F016C023F017C024F078
:109E4A0027EF4FF0120088C008F089C009F08AC0D5
:109E5A000AF08BC00BF021C00CF022C00DF023C019
:109E6A000EF024C00FF087EC4EF0500E0824146E4A
:109E7A00460E0920156E000E0A20166E000E0B20E3
:109E8A00176EA00E186E8C0E196E000E1A6E000E4A
:109E9A001B6EE2EC46F014C021F015C022F016C089
:109EAA0023F017C024F05AEF4FF01200086E81EF2A
:109EBA004FF0040E096E74EF4FF0F60E0A6E6DEF56
:109ECA004FF000F000F000F000F000F000F000F0B9
:109EDA000A2E66EF4FF074EF4FF074EF4FF0090659
:109EEA000928D8A47BEF4FF07DEF4FF062EF4FF0D7
:109EFA0081EF4FF081EF4FF008060828D8A488EFC9
:109F0A004FF08AEF4FF05EEF4FF08CEF4FF01200F8
:109F1A001B6E000E706E000E6F6EA6EF4FF09EEC79
:109F2A0019F01B507718D8B49DEF4FF09FEF4FF000
:109F3A00A6EF4FF0000EBDEF4FF0BDEF4FF0A6EFCA
:109F4A004FF01750186E196A18506F5C7050800ADB
:109F5A001A6E1950800A1A58D8A0B6EF4FF0B8EF07
:109F6A004FF094EF4FF0BAEF4FF0010EBDEF4FF004
:109F7A001200000E0001EF6F010EEE6F000E0101DC
:109F8A002C6F000E2D6F000E2E6F000E2F6F5AECE5
:109F9A004CF080928286D2EF4FF00101505151115C
:109FAA00D8B4DAEF4FF0DCEF4FF0E5EF4FF038ECD2
:109FBA0053F0000E0101516F000E506FE5EF4FF0A4
:109FCA008DEC28F0D2EF4FF0D2EF4FF007EF00F010
:109FDA0065C008F066C009F067C00AF068C00BF0F7
:109FEA00A00E0C6E8C0E0D6E000E0E6E000E0F6E15
:109FFA0087EC4EF008C014F009C015F00AC016F03C
:10A00A000BC017F088C018F089C019F08AC01AF07E
:10A01A008BC01BF02EEC3DF014C080F015C081F00F
:10A02A0016C082F017C083F0C7EC40F012007550DA
:10A03A00030DF3CF12F0F4CF13F0020E12240A6EBE
:10A04A00000E13200B6E000E0A24D96E030E0B208D
:10A05A00DA6EDF500C6E0C500E6E0D6A010E122471
:10A06A000F6E000E1320106E000E0F24D96E030E11
:10A07A001020DA6EDF50116E11500D24086E000E9A
:10A08A000E20096E49EF50F01200BD0E106EF80E48
:10A09A00116EF7EC48F04FC032F0050E336E4DC02A
:10A0AA0034F04EC035F0030E366E020EEEEC15F0AB
:10A0BA0032C04DF033C04EF067EF50F0A00E4D5E47
:10A0CA008C0E4E5AA10E4D5C8C0E4E58D8B070EFC5
:10A0DA0050F072EF50F063EF50F04DC04DF04EC0AB
:10A0EA004EF01200000102030405060B0C0D0E0FC0
:10A0FA00101113140708090A15503734313038354E
:10A10A00324E393633434F5853313437503235385B
:10A11A00303336394E53584F43434F58534E3936DE
:10A12A0033303835325037343153584F4333363958
:09A13A004E323538303134375013
:10A14400000E0C6E0001BA51D8B4ABEF50F0ADEF75
:10A1540050F0C8EF50F0DAEC51F00009D8A4B5EF94
:10A1640050F0B7EF50F0C8EF50F0DAEC51F00009BE
:10A17400D8A4BFEF50F0C1EF50F0C8EF50F0000E7C
:10A184000001BA6F010E0C6EC8EF50F00C50CBEF0B
:10A1940050F01200040E01016665D3EF50F0D5EFC4
:10A1A40050F0D9EF50F0040E666FD9EF50F066C14D
:10A1B4004EF14F6B090E0D6E000E93EC51F0C90E6B
:10A1C400106EFD0E116EF7EC48F0010E01016625CC
:10A1D400156E166A000E1622010E176E000E186E0A
:10A1E40057EC3EF0120008C00EF009C00FF00A5000
:10A1F400085C0B500958D8B002EF51F004EF51F04D
:10A204000AEF51F00AC008F00BC009F00AEF51F050
:10A2140008500C5C09500D58D8B013EF51F015EFED
:10A2240051F019EF51F00CC008F00DC009F008C04E
:10A2340008F009C009F01200156E10C00DF0155099
:10A2440093EC51F0000E176E000E166E31EF51F0C4
:10A25400200E05EC4BF0164A172A31EF51F011503D
:10A26400126E136A1250165C1750800A146E135043
:10A27400800A1458D8A041EF51F043EF51F02AEF6F
:10A2840051F045EF51F01200F2EC52F0310E106E25
:10A29400F80E116EF7EC48F0000E0D6E020E93EC02
:10A2A40051F07D0E106EFB0E116EF7EC48F00C0EA3
:10A2B400326E040E336E67C134F068C135F0FF0EA0
:10A2C400366E020EEEEC15F032C067F133C068F161
:10A2D4002AEC53F01200620E1E24D96E010E1F20C8
:10A2E400DA6EDF2A620E1E24D96E010E1F20DA6E8A
:10A2F400040EDF6480EF51F082EF51F08CEF51F0E7
:10A30400620E1E24D96E010E1F20DA6E000EDF6E5F
:10A314008CEF51F01EC01BF01FC01CF018EC4CF069
:10A3240012000F6E000E0E6E0FA09BEF51F09DEF0A
:10A3340051F0A1EF51F0400E0E26A1EF51F00FA203
:10A34400A6EF51F0A8EF51F0ACEF51F0140E0E2629
:10A35400ACEF51F081900E500D24800FD5EC4BF0F2
:10A364000FC0B7F00DC0B8F012000001D051D26F89
:10A37400D151D36FD46BD56BD21FD31FD41FD51F2C
:10A38400D22B000ED323D423D5238051D225C66FDC
:10A394008151D321C76F8251D421C86F8351D521F4
:10A3A400C96F000ECB6F000ECA6F8AEC24F0120046
:10A3B400000E80B0010E0B6E0A0E5BEC4FF080B005
:10A3C400E6EF51F0E9EF51F0010EEAEF51F0000E23
:10A3D4000B18D8A4F0EF51F0F2EF51F0DAEF51F08E
:10A3E4000B50FBEF51F0FBEF51F0DAEF51F0DAEFE5
:10A3F40051F012000B6E0BC00AF008500B5CD8B081
:10A4040006EF52F008EF52F00CEF52F008C00BF0D8
:10A414000CEF52F00B50095CD8B013EF52F015EF6B
:10A4240052F019EF52F009C00BF019EF52F00B5033
:10A434001CEF52F01200F2EC52F0370E106EFE0ECA
:10A44400116EF7EC48F06BC01BF06CC01CF067C1D8
:10A454001DF068C11EF048EC48F0C7EC40F0000E57
:10A464001C6E010E1B6E18EC4CF0000E0001A86F60
:10A47400120008C0A9FF0AC0A8FFA69EA69CA68435
:10A48400F29E550EA76EAA0EA76EA6824AEF52F050
:10A49400A1A84FEF52F051EF52F04AEF52F0A198B9
:10A4A400A694F28E1200000E0001A66F000E936FA8
:10A4B400000E926FF2EC52F0510E106EFF0E116E00
:10A4C400F7EC48F009EC00F0000E0001A16F100E4B
:10A4D400A06F1200F2EC52F0ED0E106EFE0E116E33
:10A4E400F7EC48F0A0EC48F0C7EC40F0000E1C6E0E
:10A4F400020E1B6E18EC4CF0000E0001A76F120048
:10A504007550030DF3CF0AF0F4CF0BF0010E0A24BB
:10A51400086E000E0B20096E000E0824D96E030E7F
:10A524000920DA6EDF5097EF52F0120008500A0249
:10A53400F3CF0CF0F4CF0DF008500B02F3500D26BE
:10A5440009500A02F3500D260CC008F00DC009F0A2
:10A55400ACEF52F012000001D0518025C66FD151EA
:10A564008121C76F000E8221C86F000E8321C96F3D
:10A57400000ECB6F010ECA6F8AEC24F012000101A9
:10A58400662B040E6665C9EF52F0CBEF52F0CFEFA5
:10A5940052F0000E666FCFEF52F0CCEC50F0120088
:10A5A400000E746E000E0001AD6F000EAC6F000E55
:10A5B400A16F0D0EA06FF2EC52F016EC2DF012000C
:10A5C4007550030DF3CF08F0F4CF09F0000E082402
:10A5D400D96E030E0920DA6EDF50F1EF52F012004B
:10A5E4008190010ED5EC4BF0140E5BEC4FF0000E95
:10A5F4000001B76F000EB86F1200752A000E00013B
:10A60400B26F000E106E140E116E030E1EEC51F09C
:10A61400120008C0A9FFA69EA69CA680A8CF0AF097
:10A624000A5015EF53F012001B6E1BC015F0166A8A
:10A63400030E176E010E186E57EC3EF01200000167
:10A64400E36F0001E35123EC35F03CEC27F01200FA
:10A6540069C00EF06AC00FF098EC44F01200010ECD
:0EA664000001A46F0101326933691200120077
:10EF4000000001060B0C0D10131419150F00000022
:10EF500000000000000000000000000000000000B1
:10EF600000000000000000000000000000000000A1
:10EF70000000000000000000000000000000000091
:10EF80000000000000000000000000000000000081
:10F6C0000000000000000000000000000049746518
:10F6D000726174696F6E73203F2028312D3939397A
:10F6E000290A00506F736974696F6E203F202830BB
:10F6F0002D3635356D6D290A00456E646C6F6F705F
:10F7000020776974686F7574204C6F6F700A0050B1
:10F7100072657373205B475D205768656E20526584
:10F720006164790A0053776170204C696E6561727B
:10F7300020456E61626C65203F0049732044656618
:10F7400061756C742050726F66696C65203F004C67
:10F75000696E20436C6F636B20506F6C61726974CB
:10F7600079203F00526F7420436C6F636B20506FA1
:10F770006C6172697479203F00456E61626C65202E
:10F7800050726F6772616D204D6F64653F0020207D
:10F79000202020776F726C646F66776172642E63CD
:10F7A0006F6D003C5072657373205B475D20746F12
:10F7B000205A65726F3E2000526F74617279205436
:10F7C00061626C6520446976696465720050726597
:10F7D0007373205B475D20746F2053746172740AE9
:10F7E00000526574726163742053746570205261B5
:10F7F0007465203F005377617020526F74617469A3
:10F800006F6E20446972203F00456E74657220540B
:10F810006F74616C2054656574683A0A00456E74B3
:10F820006572204E756D20446567726565733A0A8E
:10F8300000456E746572204E756D62657220446974
:10F8400076733A0A0020333E20446567202020204A
:10F85000343E20436F6E740A00202D50726573731E
:10F860002020446972656374696F6E2D004D6F646A
:10F87000653F202020202020202020202020503ADA
:10F880000020353E2047656172202020383E205000
:10F890007267726D0020353E20476561722020201E
:10F8A000393E2053657475700020383E20507267D1
:10F8B000726D2020393E20536574757000416E676B
:10F8C0006C65203F2028302D3336302E3030290A09
:10F8D000004469766973696F6E3F2028302D39398D
:10F8E0003939290A004E756D20446976733F202806
:10F8F000312D39393939290A00202D2D2D2050720A
:10F90000657373205B475D202D2D2D0A0020576104
:10F910006974696E6720666F722053454E53450ABD
:10F92000002057616974696E673A2053454E53450C
:10F930002048490A002057616974696E673A20536C
:10F94000454E5345204C4F0A00202D2D2D2063613C
:10F950006E63656C6C6564202D2D2D20004A6F67E9
:10F96000202D205B475D207768656E20646F6E6593
:10F9700000284329205374657665205761726420FE
:10F9800032303231004B6579706164204F726965A5
:10F990006E746174696F6E3A00456E61626C6520C9
:10F9A00047656172204D6F6465203F004375747434
:10F9B000657220537465702052617465203F005257
:10F9C0006F74617279205374657020526174652080
:10F9D0003F00466163746F72792044656661756C9F
:10F9E0007473203F002020202A2A2046696E697304
:10F9F000686564202A2A0A0020202A2A2043616E92
:10FA000063656C6C6564202A2A0A0020202A2A2A51
:10FA1000204C4F434B454421202A2A2A0A0020200B
:10FA20002A2A2A204C696D69742031202A2A2A0A40
:10FA30000020202A2A2A204C696D69742032202A4D
:10FA40002A2A0A0020202A2A2A2053746F707065FF
:10FA500064202A2A2A0A0020353E204C6F61642047
:10FA600020363E20536176650A0020313E205275D3
:10FA70006E202020323E20537465700A0020313EF3
:10FA8000204A6F6720202020323E204469760A00F9
:10FA90002D2D2D207375636365737366756C202D32
:10FAA0002D2D00466C697070656420546F702F4274
:10FAB0006F74746F6D005377617070656420526F5E
:10FAC000772F436F6C756D6E00466C69707065645E
:10FAD000204C6566742F5269676874004175746FB5
:10FAE00072756E2050726F6772616D203F005374A3
:10FAF00065707320506572203130306D6D203F008D
:10FB000053776170204C696E656172204469722080
:10FB10003F00456E61626C6520506F6C6172697464
:10FB200079203F005B475D20746F2073656C6563CF
:10FB300074206E65770020333E2045646974202070
:10FB4000343E204E65770A005365636F6E64732000
:10FB50003F2028312D3939290A0050726F677261B0
:10FB60006D2066696E69736865640A004368616E3A
:10FB700067652050726F66696C65203F0044697646
:10FB80006973696F6E73203D20202020200055731B
:10FB90006572207465726D696E617465640A004EE9
:10FBA0006F202844656661756C742069732000536A
:10FBB000746570732050657220333630203F0043E7
:10FBC00075747465722054726176656C203F004EC6
:10FBD000756D62657220546F204375743A0A004453
:10FBE000656772656573203D20202020202000502D
:10FBF0007265737320646972656374696F6E004522
:10FC00006E74657220436F6D6D616E643A0A0054C4
:10FC10006F6F206D616E79204C6F6F70730A0041B9
:10FC200075746F72756E205B4C6F61645D3A00573E
:10FC30006169742053656E73652048696768004583
:10FC40006E61626C652044656C6179203F002843D9
:10FC500029205374657665205761726400456E747F
:10FC600065722050726F66696C653F005370656500
:10FC700064203F2028312D35290A004375747465AE
:10FC800072204D6F76696E670A004F7574206F663B
:10FC9000206D656D6F72790A0044697265637469DD
:10FCA0006F6E20466C697000576169742053656EF1
:10FCB0007365204C6F770053657420746F20646502
:10FCC0006661756C7400506F7274313A204C696EC5
:10FCD00065617200506F7274323A204C696E6561D2
:10FCE0007200506F7274313A20526F7461727900F1
:10FCF000506F7274323A20526F746172790043759A
:10FD0000747465722054726176656C0020536C6F58
:10FD100074205B302D395D3F200044697265637447
:10FD2000696F6E204343570057616974204F7065B7
:10FD30007261746F7200496E646578696E672E2E09
:10FD40002E0A005377617020506F727473203F0049
:10FD50004E6F2053657420446976730A00446972BB
:10FD6000656374696F6E204357004C6F6F70204657
:10FD70006F7265766572004E756D20737465707371
:10FD80003A20005B475D207265736574732E0043F3
:10FD90006F6E74696E756F75733A00576169742080
:10FDA00074696D653A200041636B6E6F776C6564B2
:10FDB000676500526573657474696E670A00437500
:10FDC0007420546F6F74680A004375742052617414
:10FDD000653A20004C6F772020202D5F2D0A0048C7
:10FDE00069676820205F2D5F0A004261636B6C6168
:10FDF0007368203F00546F20437574203D200A0033
:10FE0000436F6D706C6574653A0A004C696E2053DF
:10FE1000706565642000576169742054696D6520C0
:10FE200000576169742053656E736500526F746189
:10FE30007279204A6F67004469766973696F6E3A18
:10FE400000546F74616C203D200A004C696E20479D
:10FE50006F746F200044697620476F746F20004CE8
:10FE60006F6F7020466F722000536574204469766E
:10FE7000732000466F727761726473004375747407
:10FE800065723A2000283120746F203529005072A5
:10FE90006F6772616D3A00526574726163740A0033
:10FEA000446976204164642000446567205365748A
:10FEB0002000506F732053657420004D6F766520CD
:10FEC00042792000456E64204C6F6F700056616C63
:10FED00075653A200053746172743A200059657355
:10FEE000205B205D0052657665727365004465672E
:10FEF0007265653A00546F6F74683A2000457272FB
:10FF00006F723A0A0028616E676C65290028636F7A
:10FF1000756E742900557365643A205B00467265FE
:10FF2000653A205B00526574726163740056332E2B
:10FF300030332E310052657365740A00496E646572
:10FF4000780A0054696D653A2000456D61696C3A24
:10FF50000053657475703A007374657665400044AB
:10FF600065673A202000506F733A202000476F20C9
:10FF7000746F200028736563732900476561723AC6
:10FF800000486967680A002048693A20005965738B
:10FF9000205B004469763A20005370643A200020C8
:10FFA000696E3A200052756E3A2000284A6F672920
:10FFB000004C6F61643A00536176653A0053746592
:10FFC000703A005965730A004C6F770A004C6F3A1B
:10FFD0002000206F6620004A6F673A00286D6D2967
:10FFE000004E6F0A00206D6D00286E2900456E647A
:0FFFF000004E6F70004E6F006820006D20000003
:020000040020DA
:08000000FFFFFFFFFFFFFFFF00
:020000040030CA
:0E000000FF061E1EFF0181FF0FC00FE00F4024
:00000001FF
